:100000000040002051510000915100009351000028
:1000100000000000000000000000000000000000E0
:1000200000000000000000000000000095510000EA
:1000300000000000000000009751000099510000EE
:100040009B51000071390000CD5500009B5100000C
:100050009B510000000000009B5100009B510000DC
:100060009B510000915800009B5100009B510000E3
:100070009B5100009B5100009B5100009B510000D0
:100080009B510000015A00009B5100009B51000051
:100090009B5100009B5100009B5100009B510000B0
:1000A0009B5100009B510000000000000000000078
:1000B0000000000000000000000000000000000040
:1000C00010B5064C2378002B07D1054B002B02D02E
:1000D000044800E000BF0123237010BD200400206D
:1000E0000000000000B10000044B10B5002B03D04D
:1000F0000349044800E000BF10BDC04600000000F6
:100100002404002000B10000164B002B00D1144B3A
:100110009D46402292029A1A924600218B460F4633
:100120001348144A121A08F054FD0F4B002B00D04C
:1001300098470E4B002B00D0984700200021040068
:100140000D000D48002802D00C4800E000BF08F068
:10015000FFFC2000290005F051FA08F0D3FCC0464E
:100160000000080000400020000000000000000027
:1001700020040020042800200000000000000000EF
:1001800002000120104004D1042A01D9106800099E
:1001900070470020FCE710B50400FFF7F1FF0028CE
:1001A00009D001388000031D22181279002A02D0DC
:1001B00001309842F8D110BD0122096810B51142F2
:1001C00001D0002903DA102000F082F910BD491097
:1001D000062002F017F8F9E7096810B5CB0701D53A
:1001E000002903DA102000F073F910BD4910033123
:1001F00089100022052002F005F8F6E770B50D68B9
:10020000AB0729D1042D27D90F232A684E68134044
:10021000062B0BD12800FFF7B3FF0123984201DA28
:1002200000200AE09A00AE500133F7E7052B13D106
:10023000F30703D4132000F04BF970BD7610FF2EA6
:10024000F8D82800FFF79CFF2C1D80002018A04242
:10025000E6D926700134FAE70B2000F039F9DFE720
:1002600070B50C681120E30712D54D68AB072BD190
:10027000042D29D90F262B6864101E40062E0DD19F
:10028000002C04DD2800FFF77BFFA04203DA1220D8
:1002900000F01EF901E0A400605970BD331F012B6E
:1002A00012D82800FFF76CFF8000042E02D128002E
:1002B000FFF771FF002CEADDA042E8DB01202C19DA
:1002C000E3785B001843E8E70B20E1E7F8B501238A
:1002D0000D6811201D4214D003244E6834402CD1E7
:1002E000042E2AD90F2332686D108F681340062B15
:1002F0000ED1002D04DD3000FFF742FFA84203DAE3
:10030000122000F0E5F802E0AD00AF512000F8BD8A
:10031000052B12D1002DF3DD3000FFF731FF8000F7
:10032000A842EDDB01231F4201D11320E9E77F1032
:10033000FF2FFAD87519EF70E8E70B20E1E708689E
:1003400010B5830717D1042815D90F23026813406D
:10035000062B03D1FFF714FF430004E0052B05D162
:10036000FFF70EFFC3000120184310BD042B02D17C
:10037000FFF711FFF0E70B2000F0AAF8F5E7000007
:1003800002000120104001D0501070470D22014B97
:100390001A70FAE76004002002000120104004D126
:1003A000042A01D91068000970470020FCE770B5E5
:1003B0000D000400FFF7F0FF06002800FFF7ECFF38
:1003C0000023864207D1231DB6009E1904351A006A
:1003D0009E4202D80123180070BD2978127801339B
:1003E00001358A42F3D00023F5E70000F0B585B06F
:1003F0000393019002912D4E2D4B002A02D0022230
:100400003270013A00251A601B68F554019B9D4229
:1004100001DB05B0F0BD029AAB00D058244B1C683C
:10042000C8239B0037191C1B0123184206D0214A00
:1004300043102100380008F075FF09E01E4A00282B
:1004400002D004281BD11D4A2100380008F06AFFA1
:10045000300008F0CBFF164A039B1060002B0CD035
:10046000019B013BAB4208DD154B984205D8431C6C
:100470001360202232540022F2540135C6E70428CA
:1004800010D90F2302681340042B04D101F0F6FEAB
:100490000C4A0300CDE7062B05D1FFF77DFF0A4A82
:1004A0000300C6E70123094AC3E7C04661040020F0
:1004B0008407002079A300004CA3000052A3000091
:1004C0001F03000036AA000057A3000068A3000025
:1004D000014B1870002070476004002070B501F0D7
:1004E000EFFC094C0100251D1F22280008F085FFA4
:1004F000280008F07BFF0423043080080001184323
:100500002060200070BDC0463C040020C368F0B5E8
:100510009D00836889B05D19030018330693036951
:10052000069A9F00069B0390DF19436901939B0085
:10053000D3180293CD4B1B78002B26D17F222B683A
:10054000CB491C1213409B005B58043501929F4617
:10055000039B587803F0A8FE0023039A137027E04A
:10056000C24B1B78002B10D12B68019A1C12134030
:10057000BF4A9B009B580435E9E7069B3A1DD11AF8
:10058000BA4BD82928DD1A221A70039BB74C9B68F6
:1005900021780193EA1A039B92109B7812021A4366
:1005A000039B587803F088FE0023039A237013708E
:1005B000039B069A9B680193ED1A039BAD10DD60C7
:1005C000069BFE1A039BB6101E61029B9B1A039AA0
:1005D0009B10536109B0F0BD1B783C60002B01D02B
:1005E0001700D2E72B6801991C120B40A0499B0011
:1005F0005B5817000435AAE7069B3A1DD11A9B4B9E
:10060000D82902DD1A221A70BFE728681B78291D35
:100610003860002B02D017000D00B6E76B68019917
:100620001C120B4092499B005B58170008358EE75F
:10063000069B3A1DD11A8D4BD82902DD1A221A7059
:10064000A3E7A4001B782C193C60002B01D01700F5
:100650009BE72B6801991C120B4085499B005B5856
:100660001700043573E7069B3A1DD11A7F4BD82932
:1006700002DD1A221A7088E77E49A40061581B78AF
:100680003960002B01D017007FE72B6801991C12FD
:100690000B4077499B005B581700043557E7043F30
:1006A000744B3A68A400E250704B1B78002B00D0CA
:1006B0006BE72B68019A1C1213406D4A9B009B58F4
:1006C000043544E76B4BA400E058FFF759FE043FA4
:1006D00006003868FFF754FE36180120654B760097
:1006E0000643E650614B1B78002B00D04DE72B688A
:1006F000019A1C1213405E4A9B009B58043526E762
:10070000069B3A1DD11A594BD82902DD1A221A70BC
:100710003BE70698029C0121A04202D221000C393D
:1007200009681B783960002B01D017002DE72B6872
:1007300001991C120B404E499B005B581700043571
:1007400005E7069B3A1DD11A484BD82902DD1A222B
:100750001A701AE70699029881420FD203000C3BE7
:100760001B6845495B106418E41AA40023583B60D9
:100770003E4B1B78002B05D0170006E71821197097
:100780000023F4E72B6801991C120B4038499B00A9
:100790005B5817000435DAE6069B029A934219D299
:1007A00013000C3B1B68344A043FA4185B10E31A87
:1007B000029A39689B0099502C4B1B78002B00D073
:1007C000E3E62B68019A1C121340294A9B009B58B0
:1007D0000435BCE61822254B1A70EDE7069B029AF9
:1007E00093422DD2244B3E1FE31814000C3C04937B
:1007F0002368049A5B10D31A029A9B009858FFF75B
:10080000BFFD07903068FFF7BBFD2468049B6410B0
:100810001C1B079BA4001F1801207F00029B07439D
:10082000E7503700114B1B78002B00D0ADE62B684A
:10083000019A1C1213400E4A9B009B58043586E611
:1008400018220A4B1A70EDE7069B3A1DD11A074B86
:10085000D82902DD1A221A7097E60299A40061587D
:100860001B783960002B09D017008EE66004002049
:100870004CA1000048250020FDFFFF3F2B68019997
:100880001C120B40D8499B005B58170004355EE6EC
:10089000043F029B3A68A400E250D44B1B78002B23
:1008A00000D072E62B68019A1C121340CE4A9B00BE
:1008B0009B5804354BE6029BA4001C192368043F97
:1008C00038685E10FFF75CFD36180120C74B7600D4
:1008D0001B7806432660002B00D056E62B68019A51
:1008E0001C121340C04A9B009B5804352FE6069B00
:1008F000A4003F1BBD4CBB420CD82378002B00D07A
:1009000043E62B68019A1C121340B74A9B009B5880
:1009100004351CE6B64801F025FC2378002B00D0F6
:1009200033E62B68019A1C121340AF4A9B009B5878
:1009300004350CE6A300ED18002C00DA38E6AB4BCA
:100940001B78002B00D020E62B68019A1C12134064
:10095000A54A9B009B580435F9E5043F3B68042BEE
:1009600004D1A300ED18002C00DA21E69F4B1B7880
:10097000002B00D009E62B68019A1C1213409A4AFA
:100980009B009B580435E2E5043F3B68042B06D0EE
:10099000A200AD18002C02DA002B00D108E6934B20
:1009A0001B78002B00D0F0E52B68019A1C12134035
:1009B0008D4A9B009B580435C9E53A1F13685B10AC
:1009C000013B002B06DD01215B00A4000B432D1928
:1009D0001360EDE5854B17001B78002B00D0D4E5A4
:1009E0002B68019A1C1213407F4A9B009B580435C8
:1009F000ADE53A00069B0C32D31AD82B03DD1A2240
:100A00007A4B1A70C1E5FF2361005B001940FE3B81
:100A1000FF3B1943396003990698896824120491B1
:100A20006D1A0399AD1089782D020D4302999D40EE
:100A3000091A891099401D430B43BB60039B7D60DD
:100A40009C70E4B26B4BE4000292E358039A93600B
:100A5000664A1278002A03D008331D00029F94E5ED
:100A60001D00019A9B680C351C1213405E4A9B00C6
:100A70009B58029F6BE53B1F1C68029A069B9342A2
:100A80002FD10A20E3070ED4A30715D1042C13D9C4
:100A90000F2322681340042B11D1200001F0EEFB3C
:100AA00008F0A4FC0630643003F0E8F800280FD109
:100AB000043D069B02937BE50720042CF3D0200025
:100AC000431E9841FA234042FF3318400730EAE7BB
:100AD000039B2100587803F001FC0023039A137054
:100AE000E7E7029B029A0C3B1B6803995B109B0093
:100AF000D31A0C3B1C601F1D1300083B1B685A10C7
:100B00008A70D2B23B49D2005B0055589B0A039AC7
:100B10009B009560ED18029B069A043B1B685B10D6
:100B20009B00D3180293314B1B78002B00D02CE58F
:100B30002B68019A1C1213402B4A9B009B580435CA
:100B400005E53B1F1868FFF71BFCA40006003F1BD0
:100B50001E2827DC00280DDC244B1B78002B00D03E
:100B600013E52B68019A1C1213401F4A9B009B58E7
:100B70000435ECE401F08AF9033E361801F086F9F9
:100B80001D4B801B9842F9D8184B1B78002B00D0C6
:100B9000FBE42B68019A1C121340134A9B009B58DC
:100BA0000435D4E40123039A137001F06FF9039B19
:100BB0000A3886195E60FBE43B1F1868FFF7E0FB0C
:100BC000A40006003F1B002818DC084B1B78002BF4
:100BD00000D0DAE42B68019A1C121340024A9B00F1
:100BE0009B580435B3E4C0464CA1000060040020CB
:100BF0007CA30000501D00209F860100C64B984238
:100C000003DD1D22C54B1A70BFE40123039A137044
:100C100001F03CF9FA239B005E43039B0A3E301827
:100C20005860C5E4A300FF1A002320001A00390011
:100C3000FFF7DCFBBA4EBB4C3168200003F006FA2C
:100C40003168200003F051FB3168200001F0EAFB1D
:100C5000B24B1B78002B00D097E42B68019A1C1232
:100C60001340B14A9B009B58043570E4AB4BA40081
:100C70001B783F1B002B00D087E42B68019A1C12C5
:100C80001340A94A9B009B58043560E4039803F085
:100C900059F8A24B1B78002B00D076E42B68019A00
:100CA0001C121340A04A9B009B5804354FE43B1F85
:100CB0001868002838D1083B1868C3071ED54010B3
:100CC0003A0001234100083A0B431360002859DD24
:100CD00001234200391F1A430A603A00083A126899
:100CE0001A41101A3A000C3A116819421FD0C01864
:100CF0009840A4001843029BE05027E083070FD1DF
:100D000004280DD90F2302681340062B02D1FFF7E8
:100D100043FBD5E7052B03D1FFF73EFB8000CFE770
:100D200019227E4B1A7030E440100138CEE78A0752
:100D300023D1042921D90F220E683240062A15D169
:100D4000013080004358029AA400A350734B1B78D3
:100D5000002B01D0FFF719FC2B68019A1C121340DD
:100D6000714A9B009B580435FFF7F1FB052A04D11B
:100D700008180079A4004000BCE71922674B1A70DC
:100D8000FFF703FC0435E1E7A300069AFB189B1A62
:100D9000D82B13DC0122631E002C14DC5F4B1B7864
:100DA000002B01D0FFF7F1FB2B68019A1C121340B6
:100DB0005D4A9B009B580435FFF7C9FB1A22574B2D
:100DC0001A70FFF7E2FB3A601C000437E3E7069A6B
:100DD0003B1D9B1A514ED82B03DD1A233370FFF7AE
:100DE000D4FB069B029AA40093422AD23B1F1868A8
:100DF000FFF7C6FA011E21DD029B0C3B1A68521058
:100E000082421BDB9007801A484B4018C018029B97
:100E10008000C2583B1B1A60404B3F1B1B780437B5
:100E2000002B01D0FFF7B1FB2B68019A1C12134075
:100E30003D4A9B009B580435FFF789FB2023337004
:100E4000EAE71823FBE7A3009C46FE1A002C17DCF8
:100E50001C22324B1A70002333606346FF1A2F4B5B
:100E600004371B78002B01D0FFF78FFB2B68019A0A
:100E70001C1213402C4A9B009B580435FFF767FB5C
:100E8000002033685A108300F15801230B4003D12E
:100E90000D21224A1170DFE749108A4200DD0A0065
:100EA00001308442EFDC012352001343D4E7A30056
:100EB0009C46FE1A002C17DC1C22184B1A700023CB
:100EC00033606346FF1A154B04371B78002B01D0A3
:100ED000FFF75BFB2B68019A1C121340124A9B0020
:100EE0009B580435FFF733FB002033685A1083000A
:100EF000F15801230B4003D10D21084A1170DFE79F
:100F000049108A4200DA0A0001308442EFDC0123F2
:100F100052001343D4E7C04680EE36006004002040
:100F200084070020610400204CA10000FCFFFF3F6B
:100F30003B00083B1868FFF723FA3B1F06001868C0
:100F4000FFF71EFA0023864200DA0433A4003A1B9E
:100F500017001360E34B04371B78002B01D0FFF719
:100F600014FB2B68019A1C121340DF4A9B009B580C
:100F70000435FFF7ECFA3B00083B1868FFF700FA6E
:100F80003B1F06001868FFF7FBF9F30FC217B042CA
:100F90005341A4003A1B17009B001360D14B043748
:100FA0001B78002B01D0FFF7F0FA2B68019A1C1276
:100FB0001340CD4A9B009B580435FFF7C8FA3B000D
:100FC000083B18683B1F1968A600BE1B042381421A
:100FD00002D0042802D8002333601CE00123184209
:100FE00001D01942F7D103239C461842F3D102687D
:100FF0000C331A40042AEED162461142EBD1042987
:10100000E9D90A681340042BE5D1FFF7D0F9431E54
:10101000984180003060B34BA4001B783F1B04371D
:10102000002B01D0FFF7B1FA2B68019A1C12134074
:10103000AD4A9B009B580435FFF789FA3B00083BFB
:1010400018683B1F1968A600BE1B0023814202D00E
:10105000042802D8042333601CE00123184201D085
:101060001942F7D103239C461842F3D102680C338E
:101070001A40042AEED162461142EBD10429E9D983
:101080000A681340042BE5D1FFF791F94342584118
:1010900080003060934BA4001B783F1B0437002B6B
:1010A00001D0FFF772FA2B68019A1C1213408E4A86
:1010B0009B009B580435FFF74AFA3B00083B186831
:1010C000FFF75EF93B1F06001868FFF759F9F317A1
:1010D000C20F86425341A4003A1B17009B001360C5
:1010E000804B04371B78002B01D0FFF74EFA2B689A
:1010F000019A1C1213407C4A9B009B580435FFF751
:1011000026FA3B00083B1868FFF73AF93B1F060038
:101110001868FFF735F90023864200DD0433A40088
:101120003A1B170013606F4B04371B78002B01D05C
:10113000FFF72BFA2B68019A1C1213406A4A9B0096
:101140009B580435FFF703FA3B1F1B68A400043BC0
:101150005A1E93413A1B17009B001360614B0437E2
:101160001B78002B01D0FFF710FA2B68019A1C1294
:1011700013405D4A9B009B580435FFF7E8F93B009C
:10118000083B1868FFF7FCF83B1F06001868FFF7DC
:10119000F7F832180120A4003B1B1F005200024345
:1011A0001A60504B04371B78002B01D0FFF7EDF984
:1011B0002B68019A1C1213404B4A9B009B58043524
:1011C000FFF7C5F93B00083B1868FFF7D9F83B1F4C
:1011D00006001868FFF7D4F8321A0120A4003B1B60
:1011E0001F00520002431A603E4B04371B78002B4D
:1011F00001D0FFF7CAF92B68019A1C1213403A4A32
:101200009B009B580435FFF7A2F93B00083B186888
:10121000FFF7B6F83B1F06001868FFF7B1F80200A9
:101220000120A4003B1B1F007243520002431A60BE
:101230002C4B04371B78002B01D0FFF7A6F92B6845
:10124000019A1C121340284A9B009B580435FFF753
:101250007EF93B1F1868FFF793F8061E17D11F226F
:10126000204B1A70A4003B1B1F001E601D4B04374F
:101270001B78002B01D0FFF788F92B68019A1C120C
:101280001340194A9B009B580435FFF760F93B0057
:10129000083B1868FFF774F8310005F079FE012665
:1012A00040000643DEE73B1F1868FFF769F8061E9B
:1012B0001CD11F220B4B1A70A4003B1B1F001E6089
:1012C000084B04371B78002B01D0FFF75EF92B6821
:1012D000019A1C121340044A9B009B580435FFF7E7
:1012E00036F9C046600400204CA100003B00083BDA
:1012F0001868FFF745F8310005F030FF0126490076
:101300000E43D9E73B1F1868FFF73AF8C217801859
:1013100050400122A4003B1B1F00400010431860F6
:10132000F14B04371B78002B01D0FFF72EF92B6807
:10133000019A1C121340ED4A9B009B580435FFF79D
:1013400006F9A300FE1A3068012C24D1FFF718F823
:101350000494079007F0A2FF0799002900DC0121FF
:1013600005F0FCFE049BA400C918012349001943A1
:10137000DD4B3F1B1B7831600437002B01D0FFF79A
:1013800004F92B68019A1C121340D84A9B009B5801
:101390000435FFF7DCF8FEF7F3FF04907068FEF702
:1013A000EFFF049B0130C31A0793D3E7A300FE1A93
:1013B00031002000049300F073FF049B3060FF1A9B
:1013C000C94B04371B78002B01D0FFF7DEF82B68E0
:1013D000019A1C121340C54A9B009B580435FFF725
:1013E000B6F83B00083B1868FEF7CAFF3B1F060033
:1013F0001868FEF7C5FF02000120A4003B1B1F0078
:101400003240520002431A60B74B04371B78002B5E
:1014100001D0FFF7BAF82B68019A1C121340B34AA7
:101420009B009B580435FFF792F83B00083B186877
:10143000FEF7A6FF06003B1F1868FEF7A1FF32006B
:1014400002430120A4003B1B1F00520002431A600C
:10145000A54B04371B78002B01D0FFF796F82B68BB
:10146000019A1C121340A14A9B009B580435FFF7B8
:101470006EF83B00083B1868FEF782FF06003B1F32
:101480001868FEF77DFF320042400120A4003B1B9C
:101490001F00520002431A60934B04371B78002B45
:1014A00001D0FFF772F82B68019A1C1213408F4A83
:1014B0009B009B580435FFF74AF83B1F1868FEF75E
:1014C0005FFFC0430122A4003B1B1F0040001043EC
:1014D0001860854B04371B78002B01D0FFF755F8B7
:1014E0002B68019A1C121340804A9B009B580435BC
:1014F000FFF72DF83B00083B1868FEF741FF060098
:101500003B1F1868FEF73CFF320082405100012269
:10151000A4003B1B1F000A431A60734B04371B785F
:10152000002B01D0FFF731F82B68019A1C121340F1
:101530006E4A9B009B580435FFF709F83B00083BB7
:101540001868FEF71DFF06003B1F1868FEF718FF1E
:101550003200024151000122A4003B1B1F000A433C
:101560001A60614B04371B78002B01D0FFF70DF890
:101570002B68019A1C1213405C4A9B009B5804354F
:10158000FEF7E5FF3B000C3B1868FEF7F9FE3B0059
:10159000083B06001868FEF7F3FEF1170200C317B8
:1015A000300005F02DFE3B1F049005911868FEF7F2
:1015B000E7FE02000498059905F0D6FD43000120DE
:1015C000A4003E1B37001843474B30601B7804379C
:1015D000002B01D0FEF7D9FF2B68019A1C12134093
:1015E000424A9B009B580435FEF7B1FFA300FE1A48
:1015F000310020000493FEF7DFFD049B3060FF1AEA
:10160000394B04371B78002B01D0FEF7BEFF2B6847
:10161000019A1C121340354A9B009B580435FEF773
:1016200096FFA300FE1A310020000493FEF7D4FDBC
:10163000049B3060FF1A2C4B04371B78002B01D021
:10164000FEF7A3FF2B68019A1C121340274A9B0048
:101650009B580435FEF77BFFA300FF1A39002000DA
:10166000FEF7CCFD204B1B78002B01D0FEF78DFF41
:101670002B68019A1C1213401C4A9B009B5804358E
:10168000FEF765FFA300FE1A310020000493FEF769
:10169000E7FD049B3060FF1A134B04371B78002BC7
:1016A00001D0FEF772FF2B68019A1C1213400F4AFB
:1016B0009B009B580435FEF74AFFA300FF1A390030
:1016C0002000FEF703FE084B1B78002B01D0FEF72D
:1016D0005CFF2B68019A1C121340044A9B009B5824
:1016E0000435FEF734FFC046600400204CA1000022
:1016F000A300FE1A310020000493FEF720FE049B95
:101700003060FF1AF14B04371B78002B01D0FEF735
:101710003CFF2B68019A1C121340ED4A9B009B581A
:101720000435FEF714FF069B3E1DF31AE74CD82B39
:1017300003DD1A232370FEF728FF00F0B1FB4300FE
:101740000120184323783860002B02D03700FEF7C1
:101750001CFF2B68019A1C121340DD4A9B009B580A
:1017600037000435FEF7F3FE069B3E1DF31AD74CF7
:10177000D82B03DD1A232370FEF707FF00F086FB4A
:10178000D44B400018400123184323783860002BC5
:1017900002D03700FEF7F9FE2B68019A1C121340A5
:1017A000CB4A9B009B5837000435FEF7D0FE01233F
:1017B000A600BE1B20001A003100FEF717FEC64C23
:1017C0002068643002F05AFA002802D1043DFEF786
:1017D000EFFE039B21685A78C04802F094FD012374
:1017E000039A3700137000F051FBBD4B22681B6851
:1017F000063253431818039B5860FEF7D9FEA60023
:10180000BE1B2000012300223100FEF7EFFDB24C89
:101810002068643002F032FA0028D7D0AF4802F0D6
:101820006DFBDCE7A4003E1BFEF758FE3700A74B1C
:1018300030601B780437002B01D0FEF7A6FE2B6822
:10184000019A1C121340A24A9B009B580435FEF7D4
:101850007EFEA4003E1B300000F058FB37009B4B7F
:1018600030601B780437002B01D0FEF78EFE2B680A
:10187000019A1C121340964A9B009B580435FEF7B0
:1018800066FEA4003E1B300000F042FB37008F4B89
:1018900030601B780437002B01D0FEF776FE2B68F2
:1018A000019A1C1213408A4A9B009B580435FEF78C
:1018B0004EFEA4003E1B300000F02CFB3700834B93
:1018C00030601B780437002B01D0FEF75EFE2B68DA
:1018D000019A1C1213407E4A9B009B580435FEF768
:1018E00036FEA4003F1B380000F032FB774B1B781C
:1018F000002B01D0FEF749FE2B68019A1C12134001
:10190000734A9B009B580435FEF721FEA300FE1A84
:1019100031002000049300F03BFB049B3060FF1A71
:101920006A4B04371B78002B01D0FEF72EFE2B6884
:10193000019A1C121340664A9B009B580435FEF71F
:1019400006FEA4003F1B380000F05CFB5F4B1B78D9
:10195000002B01D0FEF719FE2B68019A1C121340D0
:101960005B4A9B009B580435FEF7F1FD01212000E6
:1019700000F030FB554B1B78002B01D0FEF705FE25
:101980002B68019A1C121340514A9B009B58043546
:10199000FEF7DDFD0021200000F01CFB4B4B1B7807
:1019A000002B01D0FEF7F1FD2B68019A1C121340A9
:1019B000474A9B009B580435FEF7C9FDA4003E1B17
:1019C000300000F03BFB3700404B30601B780437A1
:1019D000002B01D0FEF7D9FD2B68019A1C12134091
:1019E0003B4A9B009B580435FEF7B1FDA4003E1B0B
:1019F000300000F037FB3700344B30601B78043781
:101A0000002B01D0FEF7C1FD2B68019A1C12134078
:101A10002F4A9B009B580435FEF799FDA4003F1BFD
:101A2000380000F0F9FA294B1B78002B01D0FEF7A3
:101A3000ACFD2B68019A1C121340254A9B009B5851
:101A40000435FEF784FDA4003F1B380002F008FFB8
:101A50001E4B1B78002B01D0FEF797FD2B68019AD7
:101A60001C1213401A4A9B009B580435FEF76FFD69
:101A7000A4003E1B300002F085FF3700134B30609E
:101A80001B780437002B01D0FEF77FFD2B68019AED
:101A90001C1213400E4A9B009B580435FEF757FD5D
:101AA000A4003F1B380002F08BFE084B1B78002B74
:101AB00001D0FEF76AFD2B68019A1C121340044AFC
:101AC0009B009B580435FEF742FDC0466004002091
:101AD0004CA10000FEFFFF7F84070020610400206E
:101AE00004000020A4003E1B300002F07FFE3700FF
:101AF000B14B30601B780437002B01D0FEF745FD59
:101B00002B68019A1C121340AC4A9B009B58043569
:101B1000FEF71DFDA300FF1A3900200000F0F6FEBD
:101B2000A54B1B78002B01D0FEF72FFD2B68019AE7
:101B30001C121340A14A9B009B580435FEF707FD79
:101B4000A300FF1A3900200000F06AFD9A4B1B78B1
:101B5000002B01D0FEF719FD2B68019A1C121340CF
:101B6000964A9B009B580435FEF7F1FCA300FF1A30
:101B70003900200000F064FD8F4B1B78002B01D052
:101B8000FEF703FD2B68019A1C1213408B4A9B0041
:101B90009B580435FEF7DBFCA300FF1A3900200038
:101BA00000F076FD844B1B78002B01D0FEF7EDFC96
:101BB0002B68019A1C121340804A9B009B580435E5
:101BC000FEF7C5FCA300FE1A31002000049302F0CA
:101BD00063FF049B3060FF1A774B04371B78002BA0
:101BE00001D0FEF7D2FC2B68019A1C121340734AF5
:101BF0009B009B580435FEF7AAFCA300FE1A310097
:101C00002000049302F050FF049B3060FF1A6A4BDF
:101C100004371B78002B01D0FEF7B7FC2B68019A24
:101C20001C121340654A9B009B580435FEF78FFC3D
:101C3000A300FE1A31002000049302F03DFF049B34
:101C40003060FF1A5C4B04371B78002B01D0FEF785
:101C50009CFC2B68019A1C121340584A9B009B580D
:101C60000435FEF774FCA300FE1A31002000049333
:101C700002F05EFD049B3060FF1A4F4B04371B7867
:101C8000002B01D0FEF781FC2B68019A1C12134037
:101C90004A4A9B009B580435FEF759FCA300FF1AE3
:101CA0003900200000F0D4FD434B1B78002B01D0FD
:101CB000FEF76BFC2B68019A1C1213403F4A9B00F5
:101CC0009B580435FEF743FCA300FF1A390020009F
:101CD00000F006FD384B1B78002B01D0FEF755FCB9
:101CE0002B68019A1C121340344A9B009B58043500
:101CF000FEF72DFCA300FE1A31002000049300F033
:101D00001BFE049B3060FF1A2B4B04371B78002B03
:101D100001D0FEF73AFC2B68019A1C121340274AA7
:101D20009B009B580435FEF712FCA300FF1A3900F4
:101D3000200000F075FD204B1B78002B01D0FEF732
:101D400024FC2B68019A1C1213401C4A9B009B58D0
:101D50000435FEF7FCFBA300FF1A3900200001F058
:101D600013FF154B1B78002B01D0FEF70EFC2B68E0
:101D7000019A1C121340114A9B009B580435FEF730
:101D8000E6FBA300FE1A31002000049301F0FCFEE4
:101D9000049B3060FF1A084B04371B78002B01D0DE
:101DA000FEF7F3FB2B68019A1C121340034A9B00B9
:101DB0009B580435FEF7CBFB600400204CA10000CB
:101DC0000023F7B55A1E0192002B07DA00F0E8FD58
:101DD00002F096F902F0BCFA642301930026300069
:101DE000194B1968B14212DD184B1A6801328A4248
:101DF0000FDAF0241A601D68154F6C43E35D002B69
:101E00001FD0E419022B06D12000FEF77FFB019BB7
:101E1000D8E70022EDE7012B0DD1002801D100F019
:101E200035F8F0226A43BB185B680A49C31A8B4233
:101E300001D80223BB54F0235D43054BEB5C022B1E
:101E4000E2D00136CCE7C046880700200000002021
:101E5000F01300209F86010000207047002070478B
:101E6000002070470020704701220020054B0649E2
:101E70001A615850043103305850083180185850B6
:101E80001A60704700800040040500000122034BE7
:101E90001A64A822D20098587047C04600800040BB
:101EA00010B5FFF7F3FFFA21890004F0E7FF10BD3A
:101EB00010B50100014803F006F910BD78130020A9
:101EC00000487047ACA300001D20704770B5054E58
:101ED0000400335C0D008B4202D003F025FD355524
:101EE00070BDC0468C07002070B50024064D635DB0
:101EF000012B05D10021200003F016FD00236355BE
:101F000001341D2CF2D170BD8C0700200D207047CC
:101F10003B207047036870B55B100120052B12D879
:101F2000094A9B009C58094D2B5D002B05D00021D0
:101F3000200003F0F9FC00232B55200003F0A2FB46
:101F400043000120184370BD94A300008C070020BB
:101F5000036870B55D101C2D14D80B4E4468735D7A
:101F6000012B05D00121280003F0DEFC012373556D
:101F7000064964108C4202DCE143C9172140280065
:101F800003F006FC70BDC0468C070020FF03000074
:101F90000B6870B55D101C2D16D80024012804DDD7
:101FA0004C68043C63425C416400094E735DA3428B
:101FB00004D02100280003F0B7FC7455280003F07A
:101FC000E7FC0423012800D00023180070BDC046A0
:101FD0008C07002070B504000D001C280ED8084E98
:101FE000335C012B04D0012103F09EFC0123335507
:101FF000290020004D1EA94103F0B4FC70BDC0466D
:102000008C07002010B543680068191F4B425941E6
:102010004010FFF7DFFF10BD37B569460A00064BD9
:1020200030CB30C203680220042B02D100F008FB41
:1020300037BD00F02DFBFBE78CA3000010B5084C6A
:102040006379002B05D00021052003F06DFC0023EF
:102050006371052003F09CFC43425841800010BD91
:102060008C07002010B5084CE37A002B05D0002126
:102070000B2003F059FC0023E3720B2003F088FCD3
:1020800043425841800010BD8C07002070477047C4
:1020900010B5034A0421034801F062FD10BDC0469B
:1020A0000800002070A90000E12110B5490209488C
:1020B00003F0E6F8FFF7D8FE0A2003F0DDFA00236C
:1020C000FF21054A995401331D2BFBD100F0B4FDCB
:1020D00010BDC046781300208C070020F8B50B4EC9
:1020E000070030000D0003F013F90400A84200DDE2
:1020F0002C003D00EB1B9C4205DD300003F012F983
:1021000028700135F6E72000F8BDC046781300209E
:1021100010B50100014803F0BBF810BD7813002092
:1021200010B5054C200003F0C1F8E1212000490260
:1021300003F0A6F810BDC04678130020064B01201E
:102140001A68064B06491A6000239A00013388502A
:10215000642BFAD17047C046B4070020AC070020BA
:102160004825002000B59BB00200054901A807F0F2
:102170000BF901A801F0DEFE02F0EAF8FCE7C04628
:1021800033A4000037B5184D04002868002801D09A
:1021900006F00CFDA400200006F0FEFC28600028DC
:1021A00002D11248FFF7DEFF01AB984207D2104B75
:1021B00002196B440193934201D20E48F2E70428BE
:1021C00002D808302860083C2B680B4A1C191360A1
:1021D0000A4B01201C60002309499A0001338850F2
:1021E000642BFAD137BDC046B4070020D9A3000044
:1021F0001CFCFFFF09A40000AC070020B007002072
:102200004825002070B50D4D0D4E04004B1C28686C
:102210009B003668C318B34203D90A20FEF758F969
:1022200070BD2B600500AB4205D80F2309011C408F
:1022300021430160F4E704C5F5E7C046AC07002080
:10224000B00700200322CB1C70B50C00D917114039
:10225000C9180500891000220420FFF7D3FF0023CE
:10226000A34206DBE343DB171C4000230419237160
:1022700070BDE95CC21811710133F1E710B5830735
:1022800006D1042804D90F2208C81340042B03D018
:102290000E20FEF71DF9014810BDC04643A4000002
:1022A00010B503240868044006D1042804D90F237C
:1022B00002681340042B03D00E20FEF709F910BD6D
:1022C000FFF7DCFF03782100233B5A4253411022E1
:1022D000C01807F029F980239B05C218044B9A42C5
:1022E00001D91420E9E7430001201843E7E7C0467D
:1022F000FFFFFF3F70B501240B680D001C4032D07A
:102300005C102000012405F0D7F8284904F0A2FF52
:1023100006F06AFB03F014FC0022254B2D6805F043
:1023200039FD002200232C4004F060FF002822D059
:10233000002C1CD06C10200005F0BEF81B4904F0E6
:1023400089FF06F051FB03F0FBFB0022184B05F060
:1023500021FD0022174B05F0F9F806F0D5FA4300ED
:102360000120184370BD0D20FEF7B2F8C9E70D201B
:10237000FEF7AEF8DFE7002C13D06C10200005F05C
:102380009BF80A4904F066FF06F02EFB03F0D8FB29
:102390000022074B05F0FEFC0022064B05F06CFF07
:1023A000DBE70D20FEF794F8E8E7C046D3023739A3
:1023B0000000D0400000E03F10B5034A022103486E
:1023C00001F0CEFB10BDC0462800002044A4000050
:1023D0000020704710B51E20FEF77AF810BD10B52A
:1023E0001E20FEF775F810BD10B51E20FEF770F820
:1023F00010BD10B51E20FEF76BF810BD10B51E20E5
:10240000FEF766F810BD10B51E20FEF761F810BD8E
:1024100010B51E20FEF75CF810BD10B51E20FEF7AB
:1024200057F810BD7047000010B5034A0921034852
:1024300001F096FB10BDC0463800002056A40000F5
:102440000120034B1860034B1B68834018437047FF
:10245000CC070020B8070020F0B5EFF3108101236E
:10246000194083F31088134C134AA4461268134E84
:10247000013A9340124F134A002B17D014680342BD
:102480000FD03D682C60C046C046C046C046C0461E
:10249000C046C046C0460C4C1568246825605B08E1
:1024A000EAE765462C6014683460F8E781F3108829
:1024B000F0BDC04608050050C80000200C050050C3
:1024C000D8070020D4070020D007002030B585B001
:1024D00001AD0C220649280006F072FB0024285D9D
:1024E00001210134FFF7F2FC0C2CF8D105B030BD0E
:1024F000E2A40000F0B585B06A463C4B3C4913802D
:102500001C2301AF93700C310922380006F058FBF0
:10251000FFF7C6FC374B384DC0182B68984201D2E4
:1025200000232B602C68002C44D13E5D012130003B
:10253000FFF7CCFC01340121300003F013FA092C21
:10254000F3D100246B461E5D01213000FFF7BEFC75
:1025500001340021300003F005FA032CF2D1C82029
:1025600080000138C046C046C046C046C046C0468E
:10257000C046C046C046C046C046C046F1D1002154
:102580000420FFF7A3FC6B4600211878FFF79EFCA0
:102590006B4600215878FFF799FC6B46002198782C
:1025A000FFF794FCFFF77CFC002413302860200028
:1025B00005B0F0BDFFF774FC2B6800249842F6D3F9
:1025C000042003F05FF80D4B0D4EC0180BD43060A3
:1025D0003068032104F0DCFC00230A4A30602B60E1
:1025E00013600124E3E73460F2E7C0461A1B0000E1
:1025F000E2A4000010270000C4070020C8FEFFFF6F
:10260000B8070020CC07002010B50124044002D0F8
:102610004410200010BD0D20FDF75AFFF9E700001F
:102620000022054B10B51A60044B1B68934201D081
:1026300002F0A8FA002010BDC80700209C1200205C
:1026400070B508680D00FFF7DFFF04006868FFF74A
:10265000DBFF621E0100042A14D8451E042D11D888
:1026600005236B439B18012215009D402B00064853
:1026700005682B430360054B1B68002B02D020002C
:1026800002F081FA002070BDC80700209C120020D3
:1026900070B508680D00FFF7B7FF04006868FFF722
:1026A000B3FF621E0100042A13D8451E042D10D862
:1026B00005236B439B1801229A4007480368934304
:1026C0000360064B1B68002B03D00022200002F0A1
:1026D0005AFA002070BDC046C80700209C12002096
:1026E000F0B5050089B008680C00FFF78DFF069073
:1026F000022D36DD6068FFF787FF0190A068FFF7C5
:1027000083FF04000127231D661E0793731C029399
:10271000079B9E4235D0052373430593019B019D82
:1027200005330493049BAB421ED0042E16D86B1EB7
:10273000042B13D80122059B2349013B5B199A40C6
:102740009446224A0B681068069A3A4003920DD0CC
:1027500062461A430A60012200280DD17F0001352C
:10276000E0E701240194CDE7029ECFE76246934360
:102770000B600028F2D0039A0299280002F003FAB5
:10278000ECE7019B1E1D042E1AD8012C18D1002540
:1027900005273B0021006B439B1999400B000A4A17
:1027A000013511689943094B11601B68002B05D056
:1027B000019B0022581D290002F0E5F9052DE8D102
:1027C000002009B0F0BDC046C80700209C120020C0
:1027D00010B5041E10DA00240A4BA400E2580123AD
:1027E0009340094A09491360094A1160094A0A4994
:1027F00011600A4A136010BDFFF766FBA042EADDD4
:10280000EAE7C04604AC0000D407002008050050E9
:10281000D8070020D00700200C05005018050050F4
:102820000200086810B5C3070DD540101823012A0F
:1028300003DD4A68042A00D10833044A1360FFF715
:10284000C7FF002010BD01204042EFE7C800002074
:102850002B4BF7B51B680C00002B03D10120404225
:10286000FFF7B6FF0126246834421AD0FF22631016
:10287000120260121040DAB21043FF221B0212044F
:10288000134018431F4B1B68202B06D1B4401E4B2E
:10289000A40EA400E35800021843FFF7DDFD00205A
:1028A000FEBD03252540FAD1042CF8D90F23226858
:1028B0001340062BF3D1FF27130901933F02019B1D
:1028C0009D42ECDA0135AB00E3583342F7D05A10A1
:1028D0005812D1B238400843FF21120209040A40BD
:1028E0001043084A1268202A06D15B009B0E064955
:1028F0009B00020258581043FFF7AEFDDFE7C046C9
:10290000D4070020C8000020D4A60000086810B535
:10291000C30703D5FFF778FE054B1860054B1B680E
:10292000002B03D0024B186802F02EF9002010BDD6
:10293000C80700209C1200200868F8B5C3071AD504
:10294000FFF762FE0300203B5E2B25D80520012205
:1029500058430023114E451DA84219D005211024CB
:10296000375C3C4200D09B180139520064100029AA
:10297000F7D10130F0E783070ED104280CD90F22DC
:1029800003681A40042A07D11B0905D00079D9E74A
:1029900001205B001843F8BD0120FCE7F7A400000C
:1029A0007FB5A04C2368002B0AD19F4A1268002AE9
:1029B00006D19E4B1B68002B01D0FFF79BFD7FBD0E
:1029C0009B4D2A68002A26D1984A1268002A1BD0FB
:1029D000FFF790FD0028F2D0FFF778FD924B2468B6
:1029E0001A681C60002A16D0002C14D101AD0C22EC
:1029F0009049280006F0E4F8285D00210134FFF733
:102A000065FA0C2CF8D1DAE7874A1268002AE5D17A
:102A1000002BE3D0E0E700211A2002F0A3FF002101
:102A20001B2002F09FFF00211C2002F09BFF2E685C
:102A3000012E5CD0022E00D1A2E0002E50D1013632
:102A40003100794C03202368994302F08BFF042066
:102A5000216801404B42594102F084FF1021236854
:102A60000A2019404B42594102F07CFF8021236823
:102A7000090119404B425941062002F073FF8021A1
:102A80002368090219404B425941072002F06AFFAE
:102A900080212368490219404B425941092002F024
:102AA00061FF80212368890219404B425941192056
:102AB00002F058FF80212368C90219404B42594156
:102AC000182002F04FFF802321681B0319404B425E
:102AD0005941172002F046FF31001A2002F042FF50
:102AE0002B680321581C04F039FB296067E7022199
:102AF0004D4C1720236819404B42594102F032FFD8
:102B000008212368182019404B42594102F02AFF3E
:102B100080212368C90019404B425941042002F02A
:102B200021FF80212368490119404B4259410A2065
:102B300002F018FF80212368C90119404B42594116
:102B4000032002F00FFF80212368890319404B42C4
:102B50005941092002F006FF802321681B04194017
:102B60004B425941192002F0FDFE3100062002F0CF
:102B7000F9FE3100072002F0F5FE31001B20ADE721
:102B80002021294C1720236819404B42594102F05B
:102B9000E9FE40212368182019404B42594102F0B8
:102BA000E1FE80212368192019404B42594102F06F
:102BB000D9FE80212368490019404B425941092020
:102BC00002F0D0FE80212368890019404B42594110
:102BD000072002F0C7FE80212368890119404B427B
:102BE0005941062002F0BEFE8021236849031940A6
:102BF0004B4259410A2002F0B5FE80212368C903E7
:102C000019404B425941032002F0ACFE8023216859
:102C10005B0419404B425941042002F0A3FE0121FC
:102C20001C205BE7C8070020C0070020CC0700205D
:102C3000BC070020E2A40000012010B54042FFF7CD
:102C4000C7FD10BD10B5034A0921034800F088FFF5
:102C500010BDC04680000020D4A7000030B502247B
:102C60008025094B094AED009C505C59002CFCD092
:102C7000A124E400884202D30021995030BD802570
:102C8000ED0018514019F5E700E00140040500008F
:102C900010B5002806D1C020B02140028902FFF7FC
:102CA000DDFF10BDB02080218002C902F7E70000DF
:102CB00043425841064B40421840B0239B02C01883
:102CC000036800201A0E532A01D11B02180A70470C
:102CD00000C0FEFF30B501248025054B054AED00FC
:102CE0009C505C59002CFCD001600021995030BDF3
:102CF00000E001400405000043425841074B4042B8
:102D00001840B0239B02C018A62310B50902DB05AA
:102D1000090A1943FFF7DEFF10BDC04600C0FEFFE1
:102D200070B5012480250D4B0D4EED009C515C5972
:102D3000002CFCD0002902DC00229A5170BD55788D
:102D400014782D0225439478013924042543D4783E
:102D5000043224062C4310C0ECE7C04600E00140DA
:102D60000405000070B505004B680A009C1C21009A
:102D7000A400FFF7D5FF281970BD0000134B1B6896
:102D8000002B0CD08022B023D2029B0200280BD152
:102D90001A1D5B681B0E522B00D110007047B02229
:102DA000C02392025B02F1E782420DD903681B0E39
:102DB000522B09D1436802339B00C018824203D9C9
:102DC00003681B0E522BE9D00020E7E7DC08002047
:102DD00070B50020FFF7D2FFFF260500002801D1C3
:102DE000280070BD03681C143440FFF7C7FFDA2CBD
:102DF000F4D10500F2E700008022F0B55200A1B046
:102E00000021674805F0E5FE802200215200654858
:102E100005F0DFFE644BFF271B681A000493534242
:102E20005A4110000592FFF733FF049C0020631EF7
:102E30009C415E4B64421C405D4BE418FFF7C8FFA9
:102E40000600002E2DD10498FFF732FF411C059893
:102E5000FFF752FF059A574D534B2C601A60FFF74E
:102E60005FF9514B64201B68A0215A4253414F4ADD
:102E70005B421340B0222C6892029B18E41A604314
:102E8000490204F085F8A0225202030000924A4948
:102E9000220007A806F078FA07A801F04BF821B045
:102EA000F0BD3268131412123A403B4003921A00EC
:102EB0000A3A092A49D83A4B039A995C002931D138
:102EC00010223E4805F085FE35002B6803991A1242
:102ED0003A40914209D11A143A400B2A27D0132ABA
:102EE0002DD00A2A01D1354B1D602800FFF746FF7F
:102EF000051EEAD1314B196800290FD02000FFF7D9
:102F000031FF04002D4B5B195968002903D02000C4
:102F1000FFF728FF040004350C2DF3D1204B0121CD
:102F2000039A99543000FFF729FF060089E73B40D8
:102F3000022BDADC214A9B00D3185D60D5E7102212
:102F400000211E4805F045FECFE71A00153A082A71
:102F5000E8D8144A0399525C002AE3D13500152BB6
:102F600000D01500300003681A143A40152A0FD01B
:102F70001D2A00D10025FFF701FF0028F3D1002D05
:102F800004D020002900FFF7EDFE0400054BC6E742
:102F9000039A1B123B409A42EDD10500EBE7C04675
:102FA000DC070020E4080020DC08002000C0FEFF51
:102FB00004C00200E00800206EA80000D82600200F
:102FC000F0B50020B7B00024FFF7D8FE27000500B9
:102FD0002600002D2ED1284D2868FFF769FE32000B
:102FE0003B0001900094254904A806F0CDF904A8FF
:102FF00000F0A0FF224B64201C682B68A0215A42DD
:103000005341204A5B421340B02292029B18E41ABB
:103010006043490203F0BCFFA02252020300009269
:103020001949220004A806F0AFF904A800F082FFB5
:1030300037B0F0BDFF226B6829689C460233FF1849
:103040000B12013613409C4200DA1C00FF200A14C8
:10305000024003926246014001920091039A0B499B
:1030600004A806F091F904A800F064FF2800FFF717
:1030700085FE0500ADE7C046DC080020E1A80000A1
:10308000E008002000C0FEFF89A80000CDA80000D5
:1030900070B50020FFF70CFE04000120FFF708FECA
:1030A000844200DA04000A4B1D686A425541280038
:1030B0001D60FFF7EDFDA0226B4252021340054A4E
:1030C00028009B18044A611C1360FFF715FE70BDB1
:1030D000DC08002004800100E0080020F8B5002092
:1030E000FFF7E6FD07000120FFF7E2FD3E00224D5D
:1030F0000643224C0DD18021C020C9024002FFF7B7
:10310000ADFD01213000FFF7F7FD1D4B2E60236060
:1031100022E0874209DD0023B0212B60184B890291
:1031200023602368002001251CE0012380212B60FF
:10313000144BC9022360F4E7120E522A0DD0002866
:1031400000D02360104C1149200006F047F9200000
:10315000FEF7AEFEFFF79CFFF8BD28005A6802326A
:1031600092009B188B4205D21A68561CE4D10028A5
:10317000F2D0CCE72160EFE7DC080020E008002077
:103180000480010004C0020024270020A4A800003D
:10319000F0B585B0039203220333DC172C4D1440A5
:1031A000E4182B682B4F5A42534180225B42D202D3
:1031B000A4103B409B18A21C0291274E9100009145
:1031C0000190316800980A1893421AD2FFF714FE52
:1031D0002B685A42534180225B421F40D202BF18E3
:1031E0003368009A9B189F420BD21C4C1C4920004C
:1031F00006F0F4F82000FEF75BFE0025280005B07D
:10320000F0BD029B356819066B461A7BA423DB05CB
:103210001343FF222F00090C1943019B12041B04C6
:10322000134019432800FFF755FD0837281D2100DA
:103230003760FFF74FFD002C04D00A9A21003800B8
:10324000FFF76EFD009B083BFF183760D6E7C046CE
:10325000DC08002000C0FEFFE0080020242700203A
:1032600047A8000010B5FFF7C7FD10BD70B59AB0B4
:10327000FFF734FFFF22254CD2000021200005F08B
:10328000A8FC0020FEF7DAFE04280ED10020FEF78D
:10329000E9FE042809D1FFF7FBFE1D4800F04AFEB5
:1032A0001C4800F047FE1AB070BD0020FFF790FDEB
:1032B000FF25002600280ED10200C300E35801308C
:1032C000591E8B41D218FF28F7D1134901A806F0E7
:1032D0005BF801A8E2E703681A142A400A2A0AD117
:1032E0001A122A40FF2A03D0D200A1180B71A05055
:1032F000FFF744FDDEE7132AFAD11B122B40FF2B08
:10330000F6D0DB00E2181671E650F1E7501D002000
:1033100016A9000026A900002EA900000021094BD3
:10332000094A59600131516059680029FCD00021D7
:103330001961012393600222044B8131FF315A50FD
:103340001A607047FC1000400010004000E100E0EF
:103350000222064B0121DA670022054B5A61054A19
:1033600011615A69002AFCD07047C04604E100E0B0
:10337000FC1000400010004010B5044C2378002BD6
:1033800001D0FFF7E5FF0020207010BDE509002007
:103390000120024B1B685B0018437047680A00203D
:1033A00000487047002700200120024B1B685B008B
:1033B000184370473C01002070B504000D00160052
:1033C000FEF76EFD8023012200215B055B6E6270BB
:1033D000E270020AA271020CE2711A0A6071637251
:1033E000000EA2721A0C1B0E26702571A17020729D
:1033F000E272237370BD0000124B10B51B68124CB3
:103400005A1C0FD0114C002B0CD0114C012B09D0A1
:10341000104C022B06D00D4C042B03D00E4C052B68
:1034200000D10B4C21000D4805F0D8FF200005F01D
:10343000DDFF0300042204339B0809481B011343EA
:10344000036010BD400100204FA9000048A9000002
:103450005AA900005FA9000054A90000EC26002032
:10346000E826002070B5214C2278002A3DD1204B5F
:1034700001215A608022D20511605A68002AFCD0CE
:10348000002207201B4B1C4901255A500439585073
:1034900008315A5019481A4958501A491A485A506E
:1034A0001A495A50A622D2009D50082218495A5053
:1034B000043158500220174958501749174858509E
:1034C000174804395850182016495850C12189000E
:1034D0005A500539FF395858921802435A50124928
:1034E000124A9950FFF71AFF257070BDE5090020B8
:1034F000FC000040001000400C050000746962757B
:103500001C05000024050000200004022C0500001A
:1035100014050000340500003C050000FFFF00001A
:103520002110010054050000E609002004050000F8
:1035300070B50E4B06001B78002B01D1FFF792FFF0
:1035400000200B4D2C7884420ED00A4B2022197893
:103550000323091B1940084B4901C918300005F025
:103560002FFB0120013C2C7070BDC046E5090020F6
:103570006C0A0020E4090020E6090020002330B591
:1035800089B0984225DD03240D682C409C4220D14F
:103590002300042D1DD90F212A681140062918D1B6
:1035A00012091F2A15D96846FFF7C2FF2300002819
:1035B0000FD06B46012218781300A04203DB6B4644
:1035C0001B5D5B0013430134A1006B50202CF3D131
:1035D0000423180009B030BD70B5414B8AB01B7888
:1035E000002B01D1FFF73EFF02AD2800FFF7A0FF3F
:1035F000002802D100200AB070BD2B780B2BF9D91E
:103600006B78012BF6D1EB78012BF3D10023354EEB
:10361000354C336023712B79344A1360002B0ED163
:10362000152169444A780B7812021A438B781B04DF
:103630001A43CB781B0613433360002318E0012B99
:1036400020D1152169444A780B7812021A438B78ED
:103650001B041A43CB781A211B06134333600E2335
:103660006A7C6944934200DD130000229A4232D101
:1036700004200021E21804339B101B010343117145
:103680002360B8E7022B03D16A7B10331621E8E7E9
:10369000042B0DD1152108226944684605F090FAE3
:1036A0000098019902F0BCF905F02EF93060C4E7EA
:1036B000052BC2D1152108226944684605F080FA1D
:1036C0000098019902F0ACF905F01EF930606A7DAE
:1036D0000A231E21C5E78D5CA01805710132C5E7DC
:1036E000E5090020680A0020002700204001002092
:1036F00010B5134B04001B78002B01D1FFF7B2FE6D
:10370000FFF726FE00200F4A0F49104B5450586017
:103710000130106058680028FCD00020186101308A
:10372000906018690028FCD0094B0A481B785B019F
:103730001B185350FFF70CFEFFF7F0FD10BDC046FD
:10374000E50900200010004004050000FC100040C6
:10375000E4090020E609002030B589B000281EDD0C
:1037600003230A6813401AD1042A18D90F201168BC
:103770000840062813D109091F2910D90124013353
:10378000990051580020214201D04910C8B26D461D
:10379000591E6854202BF2D16846FFF7A9FF00207C
:1037A00009B030BD10B5002813DD0C68E30710D553
:1037B0006410532C0DD8084B1B78002B01D1FFF758
:1037C00051FEFFF7C5FDA123044ADB00D450FFF7EB
:1037D000A5FD002010BDC046E509002000100040F6
:1037E00010B500280EDD0C68E3070BD56410FF2C24
:1037F00008D8054B1B78002B01D1FFF733FE034A95
:10380000034BD450002010BDE509002000100040FB
:103810002405000013B5002814DD0C68E30711D55A
:10382000094B64100093094B0193072C0AD8084BED
:103830001B78002B01D1FFF715FE6B46054A19577F
:10384000054BD150002016BDE2ECF0F4F8FC00046A
:10385000E5090020001000400C05000070B588B09C
:10386000002820DD0324086804401CD104281AD94C
:103870000F2302681340042B15D1FEF7FFFC06004E
:1038800005F0B4FD0500122800D912252A000221F6
:103890000D326846FFF790FD6B465D73A54205DC6F
:1038A0006846FFF725FF002008B070BD2300325D99
:1038B0006B449A730134F1E7F0B50D008BB0012829
:1038C00031DD0324086804402DD104282BD90F23AF
:1038D00002681340042B26D14B68DB0723D5FEF783
:1038E000CDFC6E6807007310019305F07FFD0500A5
:1038F0000E2800D90E252A000121113202A8FFF757
:103900005BFD6A46127902AB5A7302AA7312937373
:10391000019B76141B0ED67313745574A54205DCF7
:1039200002A8FFF7E5FE00200BB0F0BD3A5D02A94A
:1039300063189A740134F1E730B589B0002814DDBA
:103940000C68E30711D5102268460021FFF734FD0B
:103950006B466A4665105D73684663122D0E6414EB
:103960009373D4731574FFF7C3FE002009B030BD04
:10397000174B184A5968002903D0002159600131BA
:103980009160196900291FD0002018618023DB0095
:10399000D3581149012B18D1A923DB00D3585B421E
:1039A0000B600E490B78032B01D801330B700320F9
:1039B0000B490B78013303400B700A495B015B181C
:1039C000094953500123936070470860FAE7C046E5
:1039D000FC100040001000403C0100206C0A002058
:1039E000E4090020E60900200405000010B5034AA0
:1039F0000E21034800F0B4F810BDC046CC000020F2
:103A000042A90000044A05491368C85401339B05C4
:103A10009B0D13607047C046880E0020880A002066
:103A200070B5114C114A2368834202DC00232360E5
:103A300016E0155C411C2E00FA3E012E05D8994275
:103A40000FDA555C013D1F2D01D90800ECE701009C
:103A5000151A565C6E5401318B42FADC181A20603C
:103A600070BD1570FAE7C04694120020940E002035
:103A700010B5FEF70BFA064B1A68824201D90022F4
:103A80001A601B68C31A034898428041404210BD27
:103A9000840A0020204E000010B5094C094A236812
:103AA0001268934200D110BD074AD05CFEF730FB8C
:103AB0000028F8D0236801339B059B0D2360ECE7B9
:103AC0008C0E0020880E0020880A002010B504000B
:103AD000064B074A1B6812689B1ADB439B059B0D2C
:103AE000A34200DB10BDFFF7D7FFF1E7880E0020EF
:103AF0008C0E0020F7B5050056680191B000441CFB
:103B000006301700FFF7E2FFFB20FFF77BFF1C20CA
:103B1000FFF778FFE8B2FFF775FFE0B22412FFF776
:103B200071FFE0B2FFF76EFF6B461879FFF76AFF8F
:103B30000025AE4200DCF7BDAB00FB189C680135E8
:103B4000E0B2FFF75FFF2012C0B2FFF75BFF201467
:103B5000C0B2FFF757FF200EFFF754FFE9E7000060
:103B600070B5074E3368092B08DC0C255D43054C06
:103B70000133285164196160A260336070BDC04692
:103B8000900E002088270020F0B587B002900C002E
:103B9000012803DC1B20FCF79BFC45E0244B086854
:103BA0000093830709D1042807D90F230268134023
:103BB000042B02D1FEF762FB00901D4B606801935D
:103BC000830709D1042807D90F2302681340042B67
:103BD00002D1FEF753FB01900027164B1B6804939C
:103BE000049BBB42D6DD0C267E43134B0099F6188E
:103BF000306805F0E9FB051E05D17368B6680593CA
:103C0000059B9D4201DB0137EAE730680199039685
:103C100005F0DAFB0836002808D121000298039B42
:103C2000083102385B68984707B0F0BD0135E7E717
:103C300043A40000900E00208827002010B5FFF755
:103C400001F8FEF725FAFEF7B7FBFEF7EDFBFFF7ED
:103C5000CDFE00F0D9FD00F099FF10BD962210B501
:103C600012010021034804F0B4FF0022024B1A6045
:103C700010BDC046F013002088070020064B074AFD
:103C80001B6812689B1ADB439B059B0D0122834234
:103C900000DC002210007047880E00208C0E0020EF
:103CA000F8B505000C0016001F1E0ED10320FFF70B
:103CB000E5FF002808D0FA20FFF7A4FEE8B2FFF7DE
:103CC000A1FEE0B2FFF79EFEF8BD501DFFF7D6FF44
:103CD0000028F9D0FB20FFF795FEE8B2FFF792FE2F
:103CE000E0B2FFF78FFEF0B2FFF78CFE3012C0B2E9
:103CF000FFF788FE3C00E31B9E42E5DD2078FFF7DE
:103D000081FE0134F7E7000070B50024F0250B4B6D
:103D10001B68A34202DCFFF7A1FF70BD2B006343C9
:103D2000074A9B181A78002A05D0597800231120D9
:103D30001A00FFF7B5FF0134E9E7C0468807002005
:103D4000F0130020F8B507000024F0252B00634392
:103D50000C4A01349E18B74211D0317800290BD09B
:103D60000133D15C002311201A00FFF799FF2A00CC
:103D70000021300004F02DFF0A2CE7D1F8BD024BE2
:103D80001C60F9E7F013002088070020F3B5040059
:103D9000100001220300FFB00D00134013D002AB4E
:103DA0001A70431002AA02A9537042121B0E8A70A5
:103DB0000B7105220B004014C87029002000FFF78A
:103DC0006FFF7FB0F3BD032606401ED104281CD927
:103DD0000F2201680A40042A29D1022302AA137083
:103DE000FEF74CFA070005F001FBF823FF33984279
:103DF00000D91800B04202DC421C02ABDDE70136FC
:103E0000731EFB5C02AA9355F4E7042801D0002836
:103E100009D1032302AA043813704242504102AB75
:103E200058700222C9E7002ECBD10428C9D90F212E
:103E300002681140052913D1013902AE3170F82111
:103E40001209FF3192008A4200DD0A00934201DB31
:103E50000132D2E70133C118C97802AEF154F5E757
:103E60000629AED101390E00120956430196F826F3
:103E7000019FFF36B742A4DC02AE31700136934297
:103E800001DB019AE4E701270133990041583942E7
:103E90000BD03941012737700F127170B7700F14B2
:103EA000090EF77031710536E9E70149F2E7C046BE
:103EB00019FCFFFF70B502000024F0210D4E080030
:103EC000604380194578954203D001340A2CF6D11D
:103ED00070BDF022002104F07CFE074A1368013B0C
:103EE000A34200D11460002329001A001120FFF71B
:103EF000D7FEEDE7F01300208807002010B5B2B020
:103F000002236A460400137005F070FAC72800D92E
:103F1000C7200023984207DC421C6B46FE21142078
:103F2000FFF7BEFE32B010BD694601335A1EA25CD7
:103F3000CA54EFE730B5B3B002236A4605001370E8
:103F400005F054FA0400C72800D9C72400239C4276
:103F50000BDC20003230FFF7B9FD621C6B46FF21FD
:103F60001420FFF79DFE33B030BD694601335A1E61
:103F7000AA5CCA54EBE70000F7B5234B06001B68A8
:103F8000F02100930023009A9A4211DC0024F023D0
:103F90001A006243019201991C4A55182F78002F8C
:103FA00012D001340A2CF3D11948FFF7C3FF29E0DE
:103FB0000A005A43154882185078B04202D112784C
:103FC000002A1FD10133DEE7F0223900280004F077
:103FD00000FE02230D4A0199EB6053540D4AF10093
:103FE0008A58009B6E70AE70AA602F616F61A34209
:103FF00002DC054B01341C60002331001A00102044
:10400000FFF74EFEF7BDC04688070020F0130020E2
:1040100048AA0000501D002010B5FFF775FEFF24D0
:10402000084AE3005B429B18074AD35C043B012B20
:1040300003D8E043C0B2FFF79FFF013C002CEFD153
:1040400010BDC046FC070000501D0020F7B50E0053
:10405000FF247F2501901C4AE300D31A1B4A9A18BB
:104060001278062A01D0032A1DD1FF22D2009B1804
:10407000186883682B401C2B15D1C3681A002A408E
:10408000042A10D102692A40192A0CD11B0A0133D3
:104090009B000C30C018FEF7F1F8070005F0A6F9F8
:1040A0000023B04209D0013C002CD4D1F7BD019AC5
:1040B000F95CD25C9142F6D101339E42F7DCE043D9
:1040C000C0B2FFF759FFEEE7501D0020FC070000CB
:1040D00070B50500FF24084AE3005B429B18074ABD
:1040E000D35CAB4203D1E043C0B2FFF745FF013CD4
:1040F000002CF0D170BDC046FC070000501D002010
:10410000F7B5FDF7C3FE514B1A68824201D9002270
:104110001A601A684E49821A8A4200D883E01860F1
:10412000FDF7BEFE071E00D101370020FDF786FF18
:1041300001900020FDF796FF019B0090454C464DF5
:10414000002B14D02368002B00D07AE02B68276066
:10415000002B00D171E0414B01261B78002B63D16D
:104160000920FFF7B5FF3E4B1E703C4B1E70009BB5
:10417000002B12D02B68002B0FD123682F60002B4F
:104180001ED0374B01261B78002B52D10920FFF798
:104190009FFF334B1E70314B1E702368002B0FD0D6
:1041A0002F4E3278002A0BD19F4200D2276023681D
:1041B000FB1A312B04D90720FFF78AFF0123337044
:1041C0002B68002B0FD0254E3278002A0BD1BB4232
:1041D00000D92F602B68FF1A312F04D90820FFF770
:1041E00077FF012333702368002B0CD0019B002B39
:1041F00009D11B4E3378002B02D10720FFF768FF4F
:104200000023236033702B68002B0CD0009B002B05
:1042100009D1124C2378002B02D10820FFF758FF58
:1042200000232B602370F7BD0720FFF751FF0C4BD5
:104230009CE70820FFF74CFFADE7009B002B9CD1CB
:10424000ABE7009A002A95D1AAE7C046800A002071
:104250000F270000700A0020780A00207C0A002046
:10426000740A002037B500240500FFF74DFD01A8B2
:104270000194FDF7D1FE21002000FEF7D1F9FEF7F1
:104280008FFBFDF703FFFDF702FFFEF7D5FCFDF7FF
:104290002BFEA54204D0FDF751FF0248FFF74AFE6E
:1042A00037BDC04639AA0000002310B501001A002E
:1042B0001120FFF7F5FC10BD07B56B461970694674
:1042C0005A7013128B701314120ECB700A716B4656
:1042D000010005221320FFF7E3FC07BD10B50A001B
:1042E00001001220FFF752FD10BD70B50500080057
:1042F0000C003230FFF7EAFB2B00220000211B20CC
:10430000FFF7CEFC70BD10B50C00030011001420A7
:104310002200FFF7C5FC10BD70B506000020FEF7B7
:104320002DFD0024FF25002801D1200070BD036869
:104330001A142A40152A07D11B122B40B34200D170
:104340000400FEF71BFDEEE71D2AFAD10024F8E772
:10435000F0B580279DB0FFF79FFBA94CA94D2068C1
:10436000FF00391A4019FDF7B9FE23680600C3188B
:104370002360002B0ED11DB0F0BD2068391A28181B
:10438000FDF7ACFE236806001B182360FDF77EFDD9
:104390009D4B1860002EF0DC2B78FA2B00D00BE13F
:1043A0002368022B07DCFFF763FB0028E3D0012022
:1043B000FFF736FBDFE76878AC780238182823D897
:1043C00002F052FD0D1F24282B34223E68226E84F9
:1043D000D6E722222222222222222222F500FF2CAC
:1043E00012D02000FFF766FD0022884BE100CA5082
:1043F0005B181A712100130013200092FEF7C8FE0B
:1044000002E02000FFF7B8FD0320D1E72000FFF70E
:1044100051FDF9E7FFF700FEF6E7FFF775FC002016
:10442000FFF720FF7A48FFF785FDEDE7632CEBD817
:10443000784BA200D25821001520FFF7A7FCE3E734
:1044400000242000FFF768FF061E03D10134642C0E
:10445000F7D1D9E7083004F0C9FF05000530FFF7B0
:1044600035FBFB20FFF7CEFA1D20FFF7CBFAE0B2B9
:10447000FFF7C8FAE8B2FFF7C5FA2812C0B2FFF793
:10448000C1FA3700BB1B9D42E0DD387AFFF7BAFA6C
:104490000137F7E700211D2000910B000A00ADE76E
:1044A000FDF70EFD03AC5C4A642100905B4B2000DD
:1044B00004F038FF02232000237004F097FF23004C
:1044C000020000211620FFF7EBFB9DE700244F4A76
:1044D000E300D558002D28D06B689E00701DFFF7B3
:1044E000F5FA2B0000253200083321000120FFF7E8
:1044F000D7FB0020FEF742FC2F002E00002818D129
:10450000002F04D03A0001212000FFF7F3FA002D1C
:1045100004D02A0002212000FFF7ECFA002E04D07C
:10452000320000212000FFF7E5FA0134FF2CCED144
:104530006AE7FF2103681A120A40A24209D11A143D
:104540000A400B2A08D10B400CD0012B0CD0022BB7
:104550000CD0FEF713FCD1E7132AFAD100252F0067
:104560002E00F6E70600F4E70700F2E70500F0E7A3
:104570000024FFF7C9FB2200210000942300DA2069
:10458000FEF706FEFF222100D200204804F021FBA6
:104590003AE7012C02D1FEF713FD35E7022C02D1D8
:1045A000FEF760FE30E70120FFF75CFE2CE70023FA
:1045B00021001A001A2086E7FB2B00D0F7E62268BC
:1045C000042A00DCEFE62E79E878154B3602064324
:1045D0009E4200DDEBE6331D9A4200DCE3E6EB5C35
:1045E000FE2B00D0E3E66B78AC78711E1B2B6BD0F2
:1045F00018D8012B2BD0082B3DD0701DD8E6C04613
:1046000094120020940E0020840A0020501D0020E7
:104610001BAA00004825002032AA00002DAA000095
:10462000F60300001D2B60D052D31E2BE5D1012CC8
:10463000E3D10029E1DD6B79002B03D01C00322B84
:1046400000DD322464235C43344B1C60D5E7FF2C2F
:10465000D3D02000FFF72EFC6D79314AB31E0092B3
:1046600021002A000A20FEF793FD2E4BE400E050C3
:104670001B191D71C1E7632CBFD86A79022A13D0B8
:10468000032A1BD0012AB8D1E979AB790902194371
:104690002B7AA4001B0419436B7A1B060B435B00A7
:1046A0001343214AA350A8E70029A6DDB11E1C48E8
:1046B000FDF7C8FD1C4BA400E0509EE7AB79A400B9
:1046C0005A1E93419B00ECE71848FFF7BFFC94E7A4
:1046D000FF2C92D06A79022A8FD811490B200091C1
:1046E0002100B31EFEF754FD87E70B00632900DDB0
:1046F0006323002203A893420ADCD9430022C9178E
:10470000194041180A700133009021001520E9E793
:10471000A918497981540132EDE7C0460400002010
:104720009A0E0020501D002048250020990E0020E0
:104730000122094B1A60094A1368002BFCD003229E
:10474000074B1B68D8171040C0180123801006388B
:10475000400018437047C04600C0004000C1004000
:1047600008C500400120704710B5064C200000F03D
:1047700045FB0549200000F069FB0122034B1A604C
:1047800010BDC046C0120020801A060098120020FA
:1047900010B501210D20FDF799FB01210E20FDF739
:1047A00095FB00210F20FDF791FB044C200000F049
:1047B00061FA1021200000F079FA10BDA01200204B
:1047C00010B504680D20E30703D56410FF2C03D94E
:1047D0001720FBF77DFE10BDFFF7DAFFE1B20248BC
:1047E00000F086FA0020F6E7A012002010B5FFF7CF
:1047F000CFFF0021034800F07BFA4300012018435B
:1048000010BDC046A012002010B5034A072103487E
:10481000FFF7A6F910BDC046440100205DAA0000C4
:104820000D4B70B51B6804000E001500002B01D164
:10483000FFF79AFFE1B2094C200000F09EFBF1B2B5
:10484000200000F0A1FAE9B2200000F09DFA20005B
:1048500000F0FEFB70BDC04698120020C012002080
:1048600010B501240368234205D04168214202D0DB
:104870008268224203D10D20FBF72AFE10BD58109A
:10488000802801D91520F7E74910FF2901D9162002
:10489000F2E75210FF2A01D91720EDE7FFF7C0FF1A
:1048A0000020EBE7F7B501242300A0421BDD0D68D3
:1048B0002C4218D01A4B25411B684C68002B01D1A3
:1048C000FFF752FF0127174EE9B2300000F055FB09
:1048D0003C420AD03C413000E1B200F055FA3000D1
:1048E00000F0B6FB00231800FEBD03252540F6D1DD
:1048F000042CF4D90F2322681340062BEFD113099F
:104900000193019B9D42EADA0135AB00E15839423F
:10491000F7D04910C9B2300000F036FAF1E7C046CE
:1049200098120020C0120020144B70B51B680500BF
:104930000E00002B01D1FFF717FF114CEDB229003B
:10494000200000F01AFBF1B2200000F01DFA002157
:10495000200000F01DFB002801D0404270BD012264
:104960002900200000F004FB200000F0FEF90028E0
:10497000FAD0200000F0FEF9F0E7C04698120020BF
:10498000C012002010B501240368234202D0416800
:10499000214203D10D20FBF79BFD10BD581080284C
:1049A00001D91520F7E74910FF2901D91620F2E7B0
:1049B000FFF7BAFF40002043EFE70000002370B587
:1049C000344D0400EB5601330BD10D211D20FFF7B0
:1049D000ABFF5A2814D101222A212A703D38FFF753
:1049E0001FFF0023EB56022B2AD0032B49D0012BAB
:1049F0004CD121001D200124FFF796FF644225E0E1
:104A00000F211920FFF790FF332805D102235F22E1
:104A10002B7020211A38E2E70D211E20FFF784FFBA
:104A2000C7280AD1032300222A21A9382B70FFF7B7
:104A3000F7FE1B222A211E20D1E700232B70D0E78E
:104A4000012C13D129211920FFF76EFF7F2801DDEA
:104A50000138FF3803007F3301DA7F2040426423AE
:104A60007F21584302F094FA604370BD032C0BD1B0
:104A70002B211920FFF758FF043CE7E72D211920CF
:104A8000B9E721001E20B6E7052CF7D0012400204D
:104A90006442E4E77C01002010B50120FFF78EFF9F
:104AA00043000120184310BD10B50320FFF786FF17
:104AB00043000120184310BD10B50520FFF77EFF0D
:104AC00043000120184310BDF8B50123020018006F
:104AD0009A4236DD0E68334233D003244D682C40B1
:104AE0002FD1042D2DD90F2229680A40062A28D15A
:104AF000144B1B68002B01D1FFF736FEEB0704D4E3
:104B00002B681C09202C00DD20247610F1B20E4EFB
:104B10002200300000F02CFA0435A700EF19AF4254
:104B20000CD0300000F021F90028FAD0300000F05D
:104B300021F901234000184301C5F0E7012064007A
:104B40002043F8BD98120020C012002000207047BA
:104B500000207047002070470020704700207047F9
:104B600000207047002070470020704700207047E9
:104B700000207047002070470020704700207047D9
:104B800000207047704770477047000010B5034A17
:104B90000E210348FEF7E4FF10BDC046800100204F
:104BA0009EAA000010B5FDF77FFA0648FDF7EAFA65
:104BB000FFF744F80448FFF7BDF9FEF757FBFFF78E
:104BC0002BFA10BDE204000027AB000010B5FDF782
:104BD000F7F810BD70B5002504AC24780573A94220
:104BE00005D10A4B0A4A23210A4803F06DFF0160F0
:104BF0000949920052589B0002715B58A4008371CE
:104C00006358856043710223C37170BD3FAB0000E0
:104C1000A4AB00004DAB000004AC0000037B002BF4
:104C200004D143738373036101330373704700003E
:104C30001FB50191A02100240068C900D2B24450E0
:104C4000012A10D0A24209D0032A0AD0074A835071
:104C5000074B019AC250012343501FBD0222134348
:104C6000F4E70422FBE70622F9E7C04654050000FA
:104C70002405000010B50400FFF7D0FFA12223682F
:104C8000A179D20099506179064A20009950217982
:104C900004329950044B19685A689B68FFF7C8FFA3
:104CA00010BDC0460C050000B41200204BB2002B12
:104CB0000FDB80233F290FD81F290FD80F290FD8CA
:104CC00007290FD803290FD81B060168074A8B5004
:104CD000704780239B04F8E7DB04F6E71B05F4E745
:104CE0005B05F2E79B05F0E7DB05EEE72405000036
:104CF0000368074A99501A00FC32D1680029FCD099
:104D0000A321C90058580023C0B2D3607047C046E1
:104D10001C05000007B58022074BD2051A6000224F
:104D20009A6002321A710F230C3200930349023B3E
:104D30000348FFF74FFF07BDB412002000300040CA
:104D4000A0120020F8B505000E0017000024BC4298
:104D500008D02B68315D1B6828009847002801D0D7
:104D60000134F4E72000F8BD704710B51C3000F0A6
:104D7000D6F910BD10B51C3000F0C3F910BD10B548
:104D80001C3000F0D2F910BD70B5437E0D00002B31
:104D900001D1002070BD6430040000F0CFF900287C
:104DA000F7D12000290000F09DF90120F2E7000072
:104DB000F7B50193FA23002504009B0083600D4B97
:104DC0004560083303601C300F00160000F07FF9C7
:104DD0002000643000F07BF9074A2761B600B35821
:104DE00020006375019B9B009B586576A576A37593
:104DF000FEBDC046E4AB000004AC00000123A022CD
:104E0000C375837D0E49C133FF33D2059B00995092
:104E1000437DC133FF339B009950CC220169094B7C
:104E20005204CA5005220169243BCA50827D01699F
:104E30000833CA500269417D034BD1507047C046C8
:104E40000C060000240500000C050000A022002331
:104E500010B50469D200A3500A4CA1420FD90A4CE4
:104E60008C425B4109495B420B40CD21C9045B1870
:104E700004690749635005210369995010BDCC238B
:104E80005B04F5E7A086010090D00300000098FDC8
:104E900024050000F7B5040000200D0001938242B4
:104EA00065D01600402A00D9402627001C3738005C
:104EB00000F023F9B1232269DB00D55080220123C1
:104EC000216992008B50A27E002A03D122691362CD
:104ED000226913600025731EAB4207D1019B002B92
:104EE00004D0802202212369920099500122236973
:104EF0001A622369FC33DA68002A02D19A6A002A0E
:104F0000F9D09A6A002A0BD1DA60A3232269DB0068
:104F1000D1583800C9B2013500F0E4F8B542DAD30F
:104F2000019B2269002B0FD11300FC339B6A002BDD
:104F30000AD10133A376D3612369FC33DA6C002AEA
:104F4000FCD00022DA640AE000230121A37651613B
:104F50001A002369FC3399680029FCD09A60236900
:104F6000FC339A6A002A01D000229A62E8B2FEBDA0
:104F700010B50123FFF78EFF10BD0300AC3310B551
:104F800004001970643000F0B8F80123637610BD96
:104F90000023020070B5AC3243760D001178B122C7
:104FA00004000069D20081508022216992008B5058
:104FB000226901331362226993602600643630004F
:104FC00000F0ADF8002812D0300000F09AF81E4B27
:104FD0002269D0502369FC331A6A002A02D19A6AE6
:104FE000002AF9D09A6A002A01D11A62E5E72369FA
:104FF0000122002D0DD11900FC31896A002908D148
:10500000DA612369FC33DA6C002AFCD00022DA640E
:1050100007E05A612369FC339A68002AFCD0002219
:105020009A6000202369FC339A6A82420BD098620E
:105030002169064A8B588B501800022B03D0181F89
:10504000431E9841033070BD1C050000C4040000DD
:1050500010B50121FFF79CFF10BD000010B5132310
:10506000142202490248FFF7A3FE10BD0040004091
:10507000C0120020F7B506000D000C008B1801933C
:10508000019B671B9C4207D0336821781B68300066
:10509000984701340028F3D13800FEBD70B50400F4
:1050A00008000D0004F0A2F92368020029005B68E3
:1050B0002000984770BD10B50B1E02D0FFF7EEFF21
:1050C0000300180010BD10B5FFF7F5FF10BD10B5B7
:1050D00040220021040003F07CFD00232000236413
:1050E000636410BD10B53F24026C531C2340446C14
:1050F0009C4201D08154036410BD002303644364C7
:105100007047436C026C934206D03F21C25C01336E
:105110000B4043641000704701204042FBE7036CE2
:10512000406C181A00D540307047436C026C9342B3
:1051300001D0C05C704701204042FBE73F22036C76
:10514000406C01331340181A43425841C0B27047B3
:1051500003210A4802680A430260094802680A43B8
:1051600002600849084A094B9B1A03DD043BC858F2
:10517000D050FBDC00F012F8FAF7C6FF240500401F
:10518000540500400CB10000000000202004002065
:10519000FEE7FEE7FEE7FEE7FEE7FEE72D4B10B574
:1051A0001A68D2B2012A0FD12B4A126812070BD10A
:1051B0002A4AE0241168F0220800104021422DD133
:1051C0002749096811422CD01A68D2B2012A12D19B
:1051D0002149096809070ED1F020204909680140DA
:1051E000402908D11E490968014204D18020C1210B
:1051F000C005C90042501B68DBB2012B0DD1164B14
:105200001B681B0709D1154B1A68F0231A40A02A06
:105210000FD1134A12681A420ED010BD3028CFD0D9
:10522000D2E7104A104911608021104A090211602A
:10523000CAE7D02AF1D1ECE70D4B1A68012A04D055
:105240000C4A1A601A68012AFCD1C0220A4B1A6063
:10525000E3E7C046E00F00F0E40F00F0E80F00F0D5
:10526000EC0F00F004050040DFFF07C0186C0040A1
:1052700000EC06407593000014EC064001207047D6
:1052800010B503681322DB69984710BD7047000012
:10529000054B0269D1500369FC331A6A002AFCD01D
:1052A000002201201A6270471C050000030010B59F
:1052B0005C331A781F231A401E3B19009140114A93
:1052C000D167C222042104699200A150026953608F
:1052D0000269D360A02300220169DB00CA500123C8
:1052E0000169094A5B428B500169084A8B50016988
:1052F0000C3A8B50016908328B501430FFF7FDFED9
:1053000010BDC04604E100E00C05000014050000DB
:1053100010B51430FFF703FF10BD10B51430FFF7C0
:1053200004FF10BD10B51430FFF7EBFE10BD0000F8
:10533000030070B55E331A780469724BE2500300C3
:105340005D331A780469704BE250030061331C78B6
:1053500002696E4B012C00D09EE005005F352E786F
:10536000A225ED005651020060321578A12206698F
:10537000D200B5500269D4509623DB00994200D880
:105380008CE096231B01994200D88AE096235B01AA
:10539000994200D888E096239B01994200D885E085
:1053A000E1239B01994200D882E09623DB019942D8
:1053B00000D880E0E123DB01994200D87DE096230C
:1053C0001B02994200D87AE0E1231B02994200D8DF
:1053D00077E096235B02994200D874E0E1235B02F8
:1053E000994200D871E0E1239B02994200D86EE017
:1053F000474B994200D86CE0E123DB02994200D888
:105400006AE0E122002312038A425B41414A5B4287
:105410001340802252059B1801693F4A8B50A023FC
:1054200004220169DB00CA5000210369FC33D96002
:105430000369FC331962012301690B6001698B6008
:10544000C1210469890062501F215C3002780A4042
:1054500093406231314AFF315350002141560029B7
:105460003CDA0F230B40083B2D4C9B089B001B197B
:1054700003242140A140FC348C40DD69A5432C006D
:10548000C0258D4029002143D9611F23017819408F
:105490001E3B8B40136070BD00246CE79E23DB0233
:1054A000BAE79D231B03B7E71E4BB5E71E4BB3E7D7
:1054B000EC239B03B0E71D4BAEE71D4BACE71D4B48
:1054C000AAE71D4BA8E71D4BA6E71D4BA4E71D4B04
:1054D000A2E78023DB049FE71B4B9DE78C080F4B63
:1054E000A400E41803230B40FF21C025DB009940F2
:1054F000AD0066598E433100C0269E4033000B43F9
:105500006351C2E70C050000140500006C050000A3
:1055100090D0030000D0BEFE2405000000E100E0B2
:1055200000ED00E000B013000050270000A04E0086
:1055300000F0750000509D0000F0EB0000903A0173
:1055400000E0D70100B0AF0300705F07F7B500932C
:1055500008AB1B7800250193FA2304009B008360AD
:105560000E4B45600833036014300F001600FFF740
:10557000AEFD23005C3327611E70009B084A9B0030
:10558000995823005D331970019B20009B009A58A5
:1055900023005E33DD701A70FEBDC04688AC00008B
:1055A00004AC0000036910B51A00FC32D268040094
:1055B000002A0AD0A322D20099581430C9B2FFF7AA
:1055C00091FD00222369FC33DA6010BD10B502485A
:1055D000FFF7E8FF10BDC04678130020162307B57B
:1055E000022200930249013B0248FFF7AFFF07BDCB
:1055F00000200040781300207047000010B500F034
:1056000011F8FFF7F9FF012000F0ECF9FFF7CAFAF3
:10561000FFF7DCFA024B002BFAD000E000BFF7E7FF
:1056200000000000C420114B80001A58104911409E
:10563000C02212020A431A50C0218022490092025D
:105640005A501A608023A3220021DB05D200995012
:105650000122F9309A60074BFF301950C120023106
:1056600080001950403019501A60704700E100E086
:10567000FF00FFFF00100140014B18607047C0465B
:1056800038020020F7B5002320285AD8384B800074
:10569000C258042A5BD007D8022A54D055D8042314
:1056A000012A09D000234CE0062A54D051D31A2AEB
:1056B00053D002231B2AF5D12E4A116808294ED94E
:1056C00009294FD00A240226A02001252A4AC00019
:1056D00015502A482A4D07681C20BF00074029485A
:1056E000019700685759009027481B0207401F4345
:1056F000C02300989B020340FF20575157590002D6
:1057000007401F43019B1F43009B58016023184023
:1057100007433E43565101251C4B1560586800282D
:10572000FCD000205860A1230125DB00D358556030
:10573000A025ED0050511BB2A14202D015D2611A32
:10574000CB401800FEBD0823B6E71023B4E72023A2
:10575000B2E74023B0E78023AEE70123ACE708249B
:105760000026B1E70C000126AEE7091B8B40E8E7F5
:1057700004AC00003402002000700040F001002062
:1057800004050000F4010020FF00FFFFFC70004052
:10579000F0B520285BD8364B8000C258354B1E68C8
:1057A000002E30D1C227344BBF00D859334C0325CB
:1057B0000440C02000022043D851C024802064004F
:1057C000800018512E4F18602E4B803CD859FF3C5A
:1057D000A043D8510437D859A8432043D85108379B
:1057E000D8590C35A8438446072065462843D8512C
:1057F000A820C0001E50C1208026800076021E50C6
:105800001C601C4B1C60142500202B001E4C2E001D
:1058100046433659771C1BD14343E250A02303254E
:10582000C132FF329200DB05D550184B1A68082AA6
:1058300014D114234343E3189A6812485132FF32BB
:10584000920059601150DA68C1239B00C250F0BD2C
:105850009642E1D001300328D9D1F8E7082A02D9CD
:10586000083AD140E5E708239A1A9140E1E7C0469B
:1058700004AC0000DC13002000E100E0FF00FFFFAB
:105880000405000000900040F801002038020020CC
:105890002149F0B54A6C2148002A14D0A025A12640
:1058A00000230124ED05F600C258571C06D0C71886
:1058B0007F68002F02D027009740AF5114333C2B54
:1058C000F2D100234B64A0230121DB0500260F0049
:1058D0009C4614234B43C3181A1F1268104C0E4DDC
:1058E000920014195219526C002A10D01A00143A5E
:1058F0001268551C09D0103B1B68FF2B05D03B00DC
:10590000934065461A00074BEA50FC346664013147
:105910000429DED1F0BDC046FC900040F801002013
:10592000009000400C05000000B5202810D80C4A5B
:105930008000835803290BD8A0220800C133FF330D
:10594000D2059B0001F090FA020905070021D15011
:1059500000BD0C21FBE70421F9E70321F7E7C0466E
:1059600004AC000020280AD8074B8000C25801234D
:105970009340A022D205002902D104495350704718
:10598000A121C900FAE7C04604AC00000C050000E4
:1059900003000020202B0AD8A021A222C905D20092
:1059A0008858034A9B009B58D840012318407047F1
:1059B00004AC00000849094A094B10B51B68885817
:1059C000FA22190A1B0618439200002301F018FC62
:1059D0004904C00B084310BD00100140040500003D
:1059E000E013002070B5041E09D0FFF7E3FF0500A7
:1059F00000F014F8FFF7DEFF401BA042F8D370BDA3
:105A00000022044B9A60044A13680133DBB213602E
:105A10007047C046FC100140E013002070470000B2
:105A2000F0B5C64600B5CB0F9846404A4B005B0D1B
:105A30009A1882B00D000400132A2FDC002A49DBDB
:105A40003B4F17413E000E40064323D07F083900EC
:105A500029400C430AD03749BD438C4663445C421D
:105A60005C418023DB021341E4071D434146CE0025
:105A700031492B008E1922003468756820002900F6
:105A800001F064FD009001910098019922002B0023
:105A900002F0F2FB02B004BC9046F0BD332A08DDF0
:105AA0008023DB009A42F5D102000B0001F04EFD8D
:105AB000F0E7224A9446012263445242DA4002420D
:105AC000E8D052080242D1D094438022D2051A4134
:105AD0001443CBE74B005B080343DBD00B031B0BEA
:105AE0001C436342234380244D0C24031B0B23409F
:105AF0006D042B4319004346DA000F4B9B181C68BA
:105B00005D6802000B002000290001F01FFD0090DD
:105B100001910098019922002B0002F0ADFB424652
:105B20004B005B08D60733431900B3E701FCFFFFC6
:105B3000FFFF0F00EEFBFFFFB8AC0000EDFBFFFF27
:105B400030B5214A4B0087B05B0893421EDD1F4AE7
:105B5000934205DD02000B0002F08EFB07B030BD62
:105B600002AA00F035F803231840049A059B012887
:105B700013D002281DD0002814D00298039900F0F9
:105B800037FA80231B069C466144E7E70023002286
:105B90000093002300F0A6FFE0E70298039900F0CD
:105BA00027FADBE7012402980399009400F09AFF9A
:105BB000D4E7012402980399009400F093FF802316
:105BC0001B069C466144C9E7FB21E93FFFFFEF7FCD
:105BD000F0B54E464546DE465746E0B5E14B4C0033
:105BE0008FB09046894664089C4200DC87E0DE4B1B
:105BF0009C4222DCDD4A002900DC92E0DC4B02F012
:105C00003BFBDB4B06000F009C4200D17EE1D94AF2
:105C1000D94B02F031FB02000B00414630000A6014
:105C20004B60390002F028FBD34BD24A02F024FB30
:105C3000434601259860D9606BE0D04B9C4200DC64
:105C40008FE0CF4B9C4200DD55E1CE4A23159246B2
:105C50009A4451460905631A19001D00040002F018
:105C600053FE02F087FE02000B002000290008927C
:105C7000099302F001FB0022C34B02F08BF80F00E6
:105C8000060002F041FE02F075FE04000D00020065
:105C90000B00300039000A940B9502F0EDFA002257
:105CA000B94B02F077F8002200230C900D9101F01F
:105CB00079FA002800D192E1002300222000290077
:105CC00001F070FA434243410133B04A4146019228
:105CD000022208A80092524600F0A4FA4B460500A2
:105CE000002B16DA802243461206944642465B6831
:105CF000454263445360D3686344D36009E00B00BA
:105D0000020041460A604B600022002300258A60A1
:105D1000CB6028000FB03CBC90469946A246AB46EB
:105D2000F0BD934B01F012FC914B06000F009C421A
:105D300000D13DE18F4A904B01F008FC02000B00BE
:105D4000414630000A604B60390002F095FA894AFA
:105D5000894B01F0FBFB012543466D429860D960F9
:105D6000D7E700F071FF8A4A8A4B06000F0002F065
:105D700011F80022884B01F0E9FB02F0C5FD050097
:105D800002F0F8FD794A7A4B0490059102F002F88E
:105D900002000B003000390002F06EFA754A06006E
:105DA0000F0004980599744B01F0F4FF02900391E1
:105DB0001F2D00DCC7E0029A039B3000390002F07F
:105DC0005BFA83468A4653465B0024155B0DE31A53
:105DD000102B6CDD04980599D322674B520501F016
:105DE000D9FF02000B00300039000292039302F049
:105DF00043FA0A00010013000691079202003900DD
:105E0000300002F039FA029A039B02F035FA0600DC
:105E10000F0004980599614A614B01F0BBFF320005
:105E20003B0002F029FA069E079F0B000200390092
:105E300030000292039302F01FFA4B005B0D834681
:105E40008A46E41A312C32DD04980599B822544B65
:105E5000920501F09FFF03000C00020002930394DF
:105E60000B000698079902F007FA02000B000600E3
:105E70000F000698079902F0FFF9029A039B02F0BF
:105E8000FBF9484A0290039104980599464B01F0AA
:105E900081FF029A039B02F0EFF902000B00300031
:105EA00039000292039302F0E7F983468A465A4684
:105EB0005346414630000A604B60390002F0DCF97D
:105EC000029A039B02F0D8F944460B000200A2603C
:105ED000E3604B46002B00DB1BE75B46236080231F
:105EE0001B065344636080231B069C466144A060EC
:105EF000E1606D420DE70B00020002F0BDF9434680
:105F000000259860D9601860596002E7D3221A4BC7
:105F1000520502F0B1F9214A214B0D00040002F0B4
:105F2000ABF902000B00414620000A604B602900DB
:105F300002F0A2F91A4B194A02F09EF943460125D4
:105F40009860D960E5E602000B003000390002F0ED
:105F500093F96B1E154A9B009B5883468A46A342C1
:105F6000A5D130E7FB21E93F7BD902400000405436
:105F7000FB21F93F3163621A61B4D03DFB21394105
:105F8000FFFFEF7FEAFBFFFF0000704148AD00001C
:105F900083C8C96D305FE43F0000E03F7370032E9B
:105FA0008A19A33BC14920259A837B39C8AC0000DC
:105FB000D3220C4B520501F0C9FA0B4A0B4B0400DB
:105FC0000D0001F0C3FA02000B00414620000A60F8
:105FD0004B60290002F050F9034A044BB9E6032351
:105FE00073E6C04661B4D03D7370032E8A19A33B9B
:105FF000F0B54746CE4680B587B000920193754B09
:106000004F00814688467F089F4263DC02F07CFC9B
:10601000002800D1D4E04A4643464846414601F0B4
:10602000B9FE04000D006C4A6C4B01F0B3FE6C4AE3
:106030006C4B01F08BFA22002B0001F0ABFE6A4A98
:106040006A4B02F019F922002B0001F0A3FE684A06
:10605000684B01F07BFA22002B0001F09BFE664AA0
:10606000664B02F009F922002B0001F093FE644A0E
:10607000644B01F06BFA22002B0001F08BFE0290C2
:1060800003910022604B2000290001F083FE029A58
:10609000039B06000F002000290001F07BFE009A00
:1060A000019B04000D004846414601F073FE0200CA
:1060B0000B002000290002F0DFF802000B00300086
:1060C000390002F0D9F802000B0000204F4902F01D
:1060D000D3F870E002000B0001F05CFE04000D003C
:1060E0003D4A3E4B01F056FE3D4A3E4B01F02EFA32
:1060F00022002B0001F04EFE3B4A3C4B02F0BCF864
:1061000022002B0001F046FE394A3A4B01F01EFAFC
:1061100022002B0001F03EFE374A384B02F0ACF86B
:1061200022002B0001F036FE354A364B01F00EFA04
:106130002B00220001F02EFE354B029003919F426E
:106140009FDD344B00229F423DDC334900207B1809
:106150002E4916001F0002F08FF8049005910022CE
:10616000294B2000290001F015FE32003B0002F00F
:1061700083F8029A039B06000F002000290001F01B
:1061800009FE009A019B04000D004846414601F0BB
:1061900001FE02000B002000290002F06DF8020051
:1061A0000B003000390002F067F802000B00049881
:1061B000059902F061F807B00CBC90469946F0BD15
:1061C00000201249F7E7154B002604920593144F5F
:1061D000C5E7C046FFFF3F3ED43888BEE9FAA8BDF8
:1061E000C4B1B4BD9EEE213EAD529C804F7E923E26
:1061F0009015CB19A001FA3E7751C1166CC1563FDC
:106200004C5555555555A53F0000E03F0000F03F67
:106210003233D33F0000E93F0000E0FF0000E73FDA
:106220000000D23FF0B5DE464E4645465746E0B543
:10623000DC4CA5440D9114001900A49A0993DA4B83
:106240009200D6584D1E03901821E01E0696029526
:1062500000F09EFEC3430100DB1719404B1C9A005F
:106260009B1ADB001B190B9105934C1B771918D453
:10627000A59BA5009C463F1922AE6544013707E067
:10628000286802F077FB013403C60435BC4208D00D
:10629000002CF5DA00200021013403C60435BC428D
:1062A000F6D1069B002B01DA00F0FDFB069B03995B
:1062B0000133DB009A46099BDA00944600920022E3
:1062C000914672AA0492B94A6144934688469AABB1
:1062D00063449B44029B002B00DABCE15D46002630
:1062E0000027039C4D442A686B6803CC01F052FDE3
:1062F00002000B003000390001F028F9083D0600CB
:106300000F004445EFD1049B4B441E605F6008239F
:106310009C46E144D145DDD10EA804218446494282
:1063200061448C46069A93009C44614684460A91D7
:106330000399083B63448C460C93009B0092634492
:106340009B46009A0498D10003008C466344089150
:106350001E685F68002A33DD954980468C4662449A
:10636000D300984470AB9A460EAB99460022914BED
:106370003000390001F00EFD02F0C6FA02F0FAFA20
:1063800000228D4B04000D0001F004FD02000B0003
:106390003000390001F070FF02F0B6FA4B4601C33D
:1063A0009946434620001A685B68290001F0CEF840
:1063B00008235B429C46E04406000F00D045D5D13F
:1063C000059B30001A003900984600F0DDFCFF23E1
:1063D00000229B0504000D0001F0DCFC00F038FCFD
:1063E0000022764B01F0D6FC02000B0020002900B1
:1063F00001F042FF0D00040002F086FA814602F02F
:10640000B9FA02000B002000290001F035FF060058
:1064100040460F00002800DCEEE0009B18215A1EC9
:1064200092000EAB9B58091A1D000D41A9448D40E6
:106430005D1B0EAB9D5017231B1A1D41002D2DDD3A
:1064400001239C46009BE144002B00DC1CE20E9CD7
:106450000123002C00D0B5E0009A012A09D0990050
:106460000EAA54580133002C00D0ACE0009A9A4296
:10647000F5D1059B002B0EDD012B00D1A8E1022BED
:1064800009D1009B0EA95A1E92000EAB9B58079390
:106490009B029B0A8B50022D00D1C1E000230022F9
:1064A0003000390000F07EFE009B002800D194E20D
:1064B000069A591E8A4210DC414A0A9894460EAA4E
:1064C0006344944600229B0063441C68043B2243BF
:1064D0008342FAD1002A00D0C0E0069B0EAA013BFD
:1064E0009B00D358002B00D0B3E001220C9B043B4F
:1064F000596801320029FAD0009B9C466244110081
:1065000007921A0001338B4246DC0B9863468046A3
:10651000A59C4344A046099C9B00A1464A4498443C
:10652000D30022AA9146049A99449446089BA59ABE
:1065300063448446614494469A468B0063440093C6
:106540004346586802F016FA4B4618605960029BA1
:10655000002B24DB4D46039C0026002701E0286821
:1065600069680CCC01F016FC02000B003000390009
:1065700000F0ECFF083D06000F005C45EFD15346EC
:106580009E60DF6004239C460433E0449C46009BED
:10659000E144E2449845D3D1079B0093D1E600261D
:1065A0000027ECE794FDFFFF90AE000018FEFFFF10
:1065B000FFFFFF1F0000703E000070410000204000
:1065C000FFFFFF3F002180225204141B0EAA5450EB
:1065D000009999420EDD0EA884469B000EAA890000
:1065E000D25861446344CF4800E01A68821A04C359
:1065F0008B42FAD101243CE7059B002B06D1009B7E
:106600000EAA013B9B00D558ED1517E70022C64B9B
:10661000300000F0EBFD002800D024E100253DE72C
:1066200032003B000020C14901F026FE06000F00A9
:10663000002C00D132E7059A0020BC4900F0A4FBF1
:1066400002000B003000390001F016FE06000F00BA
:1066500024E7012250E70026002754E64B46059A1E
:10666000079388468B000EA9CB58183A08950592D7
:10667000002B0DD18C464146AD4B43449B006344F7
:10668000043B58680139183A0028F9D08846059229
:10669000059A0020A54900F077FB434604000D0051
:1066A000002B00DA05E29E000EAB9C464346DB0061
:1066B00066449C46059370AB9946049F67440097D7
:1066C000306802F057F922002B0001F063FB002232
:1066D00038607960974B2000290001F05BFB083F90
:1066E00004000D00043EB945EAD14AAB03939B4632
:1066F00000239A46069B424699464346013202923F
:1067000004934B46002B00DAAAE080208A4B009DC0
:106710009846C005894900260027002408E0082380
:106720009C460835E044544511DC434618685968D6
:106730002A686B6801F02EFB02000B003000390064
:1067400000F004FF013406000F00A145E7DA5B46C4
:10675000C0C39B4601239C46009BE244083B009338
:10676000029B9A45CDD1049B9846A49B022B00DD49
:106770008EE0002B37DC1FD1059B00271D00039BFB
:1067800000249C461E006544083E2A686B68380059
:10679000210000F0DBFE083D07000C00AE42F4D102
:1067A000089B002B03D080231B069C4664443A00C0
:1067B00023000D990A604B600720079B18409B231C
:1067C0009B009D443CBC90469946A246AB46F0BD1A
:1067D000009B0EA95A1E92000EAB9B5807935B02BA
:1067E0005B0A8B5057E64346002B00DA70E100202D
:1067F0000021DB004AAAD61848AF32687368083E09
:1068000000F0A4FEB742F8D1089B002B00D025E190
:106810000B0002004A984B990D9C2260636001F0C6
:106820002BFD434607000C00002B13DD01254CAE69
:10683000B14638002E0021004C4601360CCC00F049
:1068400085FEA146B045F7DA089B07000C00002B37
:1068500000D015E13A0023000D998A60CB60ABE7C8
:106860000026002773E701239C46009BE144022594
:10687000002B00DDEBE532003B0000202B4901F04E
:10688000FBFC06000F0009E60024F2E54AAB039387
:10689000A49B032B00D08FE74346002B00DC14E1C0
:1068A000039ADB009B46130091465B441E685F68B9
:1068B000234B43440293DB00994448AB9A464B4632
:1068C0005C681B681800210032003B0000900191B9
:1068D00000F03CFE04000D0002000B00009801993E
:1068E00001F0CAFC3B00320000F030FE4B469860DD
:1068F000D9601C605D6008235B429C46E144260031
:106900002F00CA45DBD14346012B00DCE3E0039AAC
:1069100013005B441E685F68029BDB0099464A4493
:10692000904610E0FFFFFF000000E03F0000F03F56
:10693000FFFFFF3F0000703E50AE0000FB21F93F1B
:10694000FFFFFF1F984643465C681B681800210044
:1069500032003B000090019100F0F8FD04000D00B2
:1069600002000B000098019901F086FC32003B0008
:1069700000F0ECFD4346039A9860D9601C605D60AE
:10698000083B26002F009A42DCD14D469446002653
:1069900000244746083565442A686B6830002100AA
:1069A00000F0D4FD083D06000C00AF42F4D1039B7B
:1069B0004A9F5D689968D868089B002B65D0802243
:1069C000120694460D9B6544604464441F605D60FC
:1069D0009960D8601E615C61EEE69A464B4607936B
:1069E000059B30005A423900089500F0CDF900228D
:1069F0003A4B06000F0000F0F9FB002824D0384B7A
:106A000000223000390001F0C5F901F07DFF524647
:106A10000400950001F0AEFF0022304B01F0BAF9FE
:106A200002000B003000390001F026FC01F06CFF81
:106A30000EAA50510122059B5244183390460593EB
:106A400093000EAAD45023E65346300039009C0030
:106A500001F05AFF0EAB1851D04619E680230D9A6B
:106A60001B06CB18106053600B0002004A984B992C
:106A700001F002FC434607000C00002B00DDD5E6C8
:106A800080231B069C466444E4E62B003A000D9DDF
:106A90002A606B600A000300AA60EB6032002300EA
:106AA0002A616B6188E6099BDB00009372AB04935B
:106AB00032E4A49B022B00DDE8E6002B00DD92E629
:106AC00000D079E6002700246AE6002600246EE75D
:106AD0000020002198E60026340068E7000070419D
:106AE0000000703EF0B5CE46474680B587B00092B4
:106AF0000193474A4B00814688465B08934207DC76
:106B00004146484601F000FF4146031E484666D014
:106B10004A4643464846414601F03CF904000D0010
:106B200002000B004846414601F034F9394A3A4B1D
:106B300006000F002000290001F02CF9374A384BDD
:106B400001F09AFB22002B0001F024F9354A364B64
:106B500000F0FCFC22002B0001F01CF9334A344BFE
:106B600001F08AFB22002B0001F014F9314B324A6C
:106B700000F0ECFC0E9B02900391002B34D00098A7
:106B8000019900222D4B01F005F9029A039B049014
:106B900005913000390001F0FDF802000B00049867
:106BA000059901F069FB22002B0001F0F3F8009A2F
:106BB000019B01F061FB224A04000D00214B3000D3
:106BC000390001F0E7F802000B002000290000F076
:106BD000BDFC02000B004846414601F04DFB07B0EA
:106BE0000CBC90469946F0BD02000B002000290025
:106BF00001F0D0F8124A134B01F03EFB32003B008B
:106C000001F0C8F84A46434600F0A0FCE7E7C0465A
:106C1000FFFF3F3E7CD5CF5A3AD9E53DEB9C2B8A0E
:106C2000E6E55A3E7DFEB157E31DC73ED561C11969
:106C3000A0012A3F1111813FA6F810110000E03F8A
:106C4000495555555555C53F49004B0819007047E2
:106C5000474AF0B54F4691464B005B0D9944464676
:106C6000D6464A46C0B505000C000E00884607000F
:106C7000132A27DC002A4BDB3E4B13419A460B00BC
:106C800052461340034318D03B4A3C4B2800210096
:106C900000F05CFC0022002300F09EFA002847D0A0
:106CA000002C04DA80234A465B031341984446468D
:106CB000534600279E43380031001CBC904699463D
:106CC000A246F0BD332A08DD8023DB009945F4D1CC
:106CD00002000B0000F03AFCEFE7294A944601223B
:106CE00063445242DA4092460242E6D0224A234BA3
:106CF0002800210000F02AFC0022002300F06CFA9A
:106D0000002815D0002C1EDB534646469F430FE05B
:106D1000194A1A4B2800210000F018FC0022002319
:106D200000F05AFA002803D0002C04DB00270026CC
:106D300038003100C1E76400640825430027002DB6
:106D4000F6D0104EF4E74B46142B0BD03422D21A57
:106D5000012393405D19BD4208D201239C462F00B8
:106D6000E044D1E7133B9C46E044CDE72F00CBE75E
:106D700001FCFFFFFFFF0F009C7500883CE4377E9D
:106D8000EDFBFFFF0000F0BF4B0070B55B0D140082
:106D90000A00002B1AD14B005B08034315D0234B8C
:106DA000002200F0F7FF224B9C422DDB0A004B0033
:106DB0005B0D363B1F4DE318AB422ADC002B0DDD8B
:106DC0001D4C1B0522401A43110070BD1B4DAB42E8
:106DD000F0D102000B0000F0B9FBF6E71D003535DD
:106DE00019DA174B02009C4209DD0B0015481649C1
:106DF00000F032F8134A144B00F0CCFFE5E70B002B
:106E00001248134900F028F8104A114B00F0C2FF55
:106E1000DBE70200E9E7084C363322401B05134349
:106E2000190000220B4B00F0B5FFCEE700005043E5
:106E3000B03CFFFFFE070000FFFF0F80FF070000D0
:106E400050C300009C7500883CE4377E59F3F8C2BB
:106E50001F6EA5010000903C30B54A00DB0FDB0738
:106E600052081A43110030BD02B471464908490066
:106E7000095C49008E4402BC7047C04600224308AA
:106E80008B4274D303098B425FD3030A8B4244D3F2
:106E9000030B8B4228D3030C8B420DD3FF22090234
:106EA00012BA030C8B4202D31212090265D0030BF3
:106EB0008B4219D300E0090AC30B8B4201D3CB03E9
:106EC000C01A5241830B8B4201D38B03C01A52412B
:106ED000430B8B4201D34B03C01A5241030B8B422D
:106EE00001D30B03C01A5241C30A8B4201D3CB0218
:106EF000C01A5241830A8B4201D38B02C01A5241FD
:106F0000430A8B4201D34B02C01A5241030A8B42FF
:106F100001D30B02C01A5241CDD2C3098B4201D317
:106F2000CB01C01A524183098B4201D38B01C01A95
:106F3000524143098B4201D34B01C01A524103090C
:106F40008B4201D30B01C01A5241C3088B4201D3BB
:106F5000CB00C01A524183088B4201D38B00C01A68
:106F6000524143088B4201D34B00C01A5241411A8F
:106F700000D20146524110467047FFE701B500209C
:106F800000F0F0F802BDC0460029F7D076E7704760
:106F900003460B437FD4002243088B4274D303097A
:106FA0008B425FD3030A8B4244D3030B8B4228D31B
:106FB000030C8B420DD3FF22090212BA030C8B4241
:106FC00002D31212090265D0030B8B4219D300E0E1
:106FD000090AC30B8B4201D3CB03C01A5241830B66
:106FE0008B4201D38B03C01A5241430B8B4201D316
:106FF0004B03C01A5241030B8B4201D30B03C01A3F
:107000005241C30A8B4201D3CB02C01A5241830AB8
:107010008B4201D38B02C01A5241430A8B4201D3E7
:107020004B02C01A5241030A8B4201D30B02C01A11
:107030005241CDD2C3098B4201D3CB01C01A524178
:1070400083098B4201D38B01C01A524143098B4201
:1070500001D34B01C01A524103098B4201D30B01EA
:10706000C01A5241C3088B4201D3CB00C01A52410F
:1070700083088B4201D38B00C01A524143088B42D4
:1070800001D34B00C01A5241411A00D2014652416D
:10709000104670475DE0CA0F00D04942031000D38C
:1070A0004042534000229C4603098B422DD3030AE1
:1070B0008B4212D3FC22890112BA030A8B420CD3F1
:1070C000890192118B4208D3890192118B4204D31A
:1070D00089013AD0921100E08909C3098B4201D39A
:1070E000CB01C01A524183098B4201D38B01C01AD4
:1070F000524143098B4201D34B01C01A524103094B
:107100008B4201D30B01C01A5241C3088B4201D3F9
:10711000CB00C01A524183088B4201D38B00C01AA6
:107120005241D9D243088B4201D34B00C01A52417D
:10713000411A00D20146634652415B10104601D30A
:107140004042002B00D54942704763465B1000D394
:10715000404201B5002000F005F802BD0029F8D03A
:1071600016E770477047C046D0400B1C1141203ACB
:1071700003D49C461341184363465242934018433C
:107180007047C0468446101C62468C46191C6346F4
:1071900000E0C0461FB500F095FD002801D4002195
:1071A000C8421FBD10B500F0EDFC4042013010BDDB
:1071B00010B500F087FD002801DB002010BD012084
:1071C00010BDC04610B500F07DFD002801DD002097
:1071D00010BD012010BDC04610B500F00FFD002805
:1071E00001DC002010BD012010BDC04610B500F02C
:1071F00005FD002801DA002010BD012010BDC046A9
:10720000F0B5CE46474615042D0C2E0080B5070478
:10721000140C3F0C9946030C7E435D436743634364
:107220007F19340CE4199C46A54203D980235B02E4
:107230009846C4444B4643435143250C36046544A9
:10724000360C2404A4195B19591820000CBC904674
:107250009946F0BDF0B54E4657464546DE46E0B588
:1072600043025B0A450083B00F1C99462D0EC60FE2
:10727000002D57D0FF2D24D08020DB00C004184300
:10728000002381469A469B467F3D7C027A00FB0F95
:10729000640A120E984623D0FF2A4BD0E3008024C4
:1072A0000020E4047F3A1C43AD186B1C4746019351
:1072B000534677403A000F2B48D87D499B00CB5866
:1072C0009F46002B00D085E008339A46063B9B463C
:1072D0007C027A00FB0FFF25640A120E9846DBD170
:1072E000002C00D090E0524601231A439246012020
:1072F000DBE74C4658461700022824D0032800D16B
:10730000CFE00022002301284DD15802D205400AC7
:10731000FF071043384303B03CBC90469946A24651
:10732000AB46F0BD002B5BD104239A46033B0025FE
:107330009B46AAE7FF35002C60D1524602231A4330
:1073400092460220B1E7FF220023DEE74B461B0CEA
:107350009C464B462604360C180461463300220C2A
:107360006446000C43434E435043544380191A0C67
:107370001218964203D9802149028C4664441B04AA
:107380001B0C1004C01883015E1EB341800E18430D
:10739000130C1B199B0103431C00230179D5012306
:1073A00062081C401443019A7F32002A4DDD6307B6
:1073B00004D00F232340042B00D00434230103D531
:1073C0003C4B019A1C408032FE2ABCDCA3015B0AC4
:1073D000D2B29AE70C239A46093BFF259B4654E715
:1073E000180001F053FB4A46431F76259A400023BC
:1073F0006D4291462D1A9A469B4646E75246032314
:107400001A439246032050E7200001F03FFB431F40
:107410002D1A9C40763D002047E780230027DB03A0
:10742000FF2272E7424666E74C463200584662E762
:1074300080234A46DB031A4222D01C4220D1234338
:107440005B025B0A4746FF225FE701239A1A1B2A69
:1074500021DC23000199D3409E318C401A00230087
:107460005C1EA34113435A0704D00F221A40042A7A
:1074700000D004335A0111D49B015B0A002244E777
:1074800080234A46DB0313435B025B0A3700FF227B
:107490003BE7019587E70022002336E7012200231E
:1074A00033E78023DB0323435B025B0AFF222CE7E5
:1074B000A0AE0000FFFFFFF770B500283DD0C31756
:1074C000C5185D40C40F280001F0E0FA9E22121A90
:1074D000962A07DCD2B2082833DD083885406802D6
:1074E000400A23E0992A0BDD052329001B1AD94005
:1074F00003001B339D402B005D1EAB4119430D0063
:10750000052801DD431F9D402B000F490B406E07EE
:1075100009D00F263540042D05D004335D0102D576
:107520009F220B40121A9B01580AD2B24002D20588
:10753000400AE4071043204370BD002400220020CD
:10754000F4E76802400AF1E7FFFFFFFBF0B54F46A2
:107550004646D6460C000903C0B5490A470F5E00EF
:1075600039431F03DB0F9C4665007B0A570F1F43FF
:107570006D0DE40F760DA146C000B846D200AB1BDE
:1075800064457BD0002B5FDD002E00D0A4E03E00E0
:10759000164300D112E15E1E002E00D09EE1871A34
:1075A0004346B84280410125C91A4042091A0B02DC
:1075B00000D431E149024E0A002E00D16EE13000C4
:1075C00001F064FA0300083B1F2B00DD61E120227B
:1075D0003900D21A9E40D1409F400E439D4200DDAB
:1075E00051E15D1B6B1C1F2B00DD7CE12021C91AC2
:1075F0003D0030008F408840DD40791E8F413100D2
:1076000007222843D940002507433A40002A09D0E1
:107610000F233B40042B05D03B1DBB42BF417F42A3
:10762000C9191F000B0200D426E26A1CC64B55057F
:107630006D0D9A4200D106E1C44AFF080A40530783
:1076400052023B43120B8EE0002B00D0B8E06B1CC3
:107650005B055B0D012B00DC30E1871A4346B84225
:10766000B641CB1A76429E1B330200D54CE13B005B
:107670003343A1D100220024002570E0002B00DC60
:10768000E5E0002E00D183E0AF4EB54260D0802609
:1076900036043743B846382B00DC3EE143461343FB
:1076A0001F007A1E97413F188742804140420918C7
:1076B0000B0200D4B0E0A44B01359D4200D1C3E0E1
:1076C000A24A7B080A4001210F401F435108D307FB
:1076D00007221F433A4099E79B4EB54238D0802697
:1076E00036043743B846382B00DDDCE01F2B00DCC6
:1076F00030E11E004746203EF740BC46202B04D018
:107700004026F31A46469E403243170063467A1ECF
:1077100097411F43CCE0002B00D104E243461343C2
:1077200000D159E14B07C00818438023C9081B0347
:10773000194208D04546ED081D4204D14346D00801
:10774000590708432900420FC9007F4D1143C0006B
:107750004B07CA087C49C00803438D4268D0120316
:107760006D05120B6D0D002112031800130B0A0D8D
:1077700012051A43764B2D0513402B435B00E4079B
:107780005B08234319001CBC90469946A246F0BDF5
:107790003E00164312D05E1E002E00D000E1871876
:1077A0008742804141444042091801250B0233D5EC
:1077B000022585E764463300414610001D00C7E7F7
:1077C000002D00D0DAE00C000443F3D05C1C00D1A3
:1077D0009FE15D4CA64200D12FE1DB43382B00DD59
:1077E00066E11F2B00DD83E120240500E41A0F0071
:1077F000DD40D940A0404346A7405B1A441EA0414B
:1078000098462F433843171ABA4292414346524290
:10781000991A64463500CAE607223A40002A00D089
:10782000F6E64B07CA084849FF083B438D4296D10C
:107830001900114300D19EE1802109030A4312037C
:10784000120B414D8FE71500002200238BE7002B20
:1078500000D0C7E06B1C5F057F0D012F00DCF1E05D
:10786000394DAB4200D1B9E085180A008542894103
:107870004244494251180722CF076D082F43490857
:107880003A401D00C2E607223049ED1A31403A4025
:10789000BCE63E002838864000279FE6380001F00D
:1078A000F5F820308EE6434613431F007A1E9741B9
:1078B000C71BB84280414042091A78E60E003B00DF
:1078C00006431343002D61D1002E00D0F4E0002BBD
:1078D00000D11BE164463900100039E71A4FBB4262
:1078E0007AD03300FFE630001F3DE840202B03D064
:1078F0004021CB1A9E4037437B1E9F4107220743FE
:107900003A400021002589E7171A4346BA42B6419A
:10791000591A76428E1B64464EE61F2B00DDADE001
:1079200020264746F61AB740B9461700B246DF4050
:107930004E463E4337005646B240561EB2411743AC
:107940004246DA408918AEE6FF070000FFFF7FFFDE
:10795000FFFF0F8020264746F61AB740B9461700AA
:10796000B246DF404E463E4337005646B240561EB2
:10797000B24117434246DA40891A99E77F4CA64242
:107980005BD0802424045B42214327E7002E0CD1E6
:10799000002B00D1CBE0644639001000774DD7E6CC
:1079A000764FBB4218D0330075E6002B14D04B073E
:1079B000C00818438023C9081B03194207D0FC08DC
:1079C0001C4204D17907D0080843E14621004C4607
:1079D000420FC9001143C000684DB9E61D000022E6
:1079E0000023C0E6002D5BD10D00054300D1E2E687
:1079F0005D1C00D1B0E0614DAE421FD0DB43382B9F
:107A000071DC1F2B00DD96E020250F00ED1AAF4042
:107A1000B9460700AA46DF404D463D432F00554674
:107A2000A840D940451EA84188440743BF18974243
:107A300092415142414435003AE6644635004146A0
:107A4000100085E60B000343002D00D063E6002BF9
:107A5000F5D04346134300D17AE687188742804128
:107A600007224144404209183A400B0200D4D5E6AF
:107A7000434B01351940C9E5380069E61E00474609
:107A8000203EF740BC46202B04D04026F31A464641
:107A90009E403243170063467A1E97411F4302E619
:107AA000364DAE42CAD080252D045B422943A6E75D
:107AB0000843411E8841A6E6002B00D148E6871AFC
:107AC0004346B842B641CB1A76429E1B33024BD591
:107AD000171A4346BA429241591A5242891A07224A
:107AE00064463A4092E501430F00791E8F419DE7BD
:107AF0001C000F00203CE740202B03D04024E31A59
:107B000099400843411E884138437CE60022002406
:107B100025E6171A4346BA429241591A5242891A27
:107B20006446350043E541461000144D10E68022BE
:107B30000024120380E61D000F00203DEF40BC46EC
:107B4000202B03D04025EB1A9940084307006346D9
:107B5000781E87411F4369E7871897429B4141443C
:107B60005B42C9183500A3E53B003343CED0072262
:107B700031003A4052E600231A00F4E5FF07000006
:107B8000FFFF7FFFF0B54F464646D6468446C0B558
:107B90008046194E18030F034D00000B5C0082460F
:107BA0003F0B6D0DC90F9146640DDB0F0120B542EF
:107BB0000AD0B44203D0A54201D157450CD01CBC19
:107BC00090469946A246F0BD66463E43F7D1AC4288
:107BD000F5D154461443F2D10120C845EFD1994262
:107BE00007D0002DEBD163461F433800471EB84134
:107BF000E5E70020E3E7C046FF070000F0B54F4689
:107C00004646D6464D00C0B50E03C90F8A462C49DC
:107C10001F035C008046360B6D0D91463F0B640DD3
:107C2000DB0F8D421ED08C4216D0002D1ED130436A
:107C30008446002C01D13A4323D06246002A1AD050
:107C40009A4529D0514602200139084001381CBC10
:107C500090469946A246F0BD39001143E5D0022076
:107C60004042F4E73043FAD1AC420FD0002C0FD1A0
:107C70003A43E7D00CE00122013B93431800013066
:107C8000E5E763460020002BE1D0DBE73A43E6D18D
:107C90009A45D7D1A542D5DCA54205DBBE42D1D855
:107CA00008D00020BE42D2D250460123013898436A
:107CB0000130CCE7C845C5D80020C845F4D3C6E795
:107CC000FF070000F0B54F464646D6464D00C0B50A
:107CD0000E03C90F8A462E491F035C008046360BEF
:107CE0006D0D91463F0B640DDB0F8D4218D08C4219
:107CF00011D0002D18D130438446002C1ED13A43B8
:107D00001CD163460020002B30D05146022001399F
:107D1000084001382AE039001143EAD0022025E06A
:107D20003043FBD1AC4226D0002C26D13A4324D19B
:107D30005146022001390840013817E06246002A06
:107D40000FD09A45E1D1A54205DBBE42DDD819D05E
:107D50000020BE420AD25046012301389843013028
:107D600004E00122013B9343180001301CBC904603
:107D70009946A246F0BD3A43D0D19A45C5D1A54215
:107D8000C3DCE0E7C845C0D80020C845E3D3EDE731
:107D9000FF070000F0B55746DE464E464546E0B5C3
:107DA000834606000F03480087B092461D003F0B34
:107DB000400DCC0F002800D16FE0DE4B984238D048
:107DC0008023FF001B041F43730F3B430193DA4BD7
:107DD0000027994600239B46F60081442B03690047
:107DE0001B0B52469846490DED0F002900D185E046
:107DF000D04B994200D173E04346DA0080231B0444
:107E000013435246CC48520F844613435246002037
:107E10006144D20089442100694000918C460121CF
:107E200049448A460F2F00D990E0C449BF00CF597A
:107E3000BF465B463B43019300D06AE1022308271B
:107E4000002681469B46C9E732005846019B6146A1
:107E50000091022800D175E0032800D1FEE101283D
:107E600000D02CE100230027002600253F032A0D27
:107E70003F0BB34812053A4302401B051343009AD7
:107E80005B00D1075B080B433000190007B03CBC16
:107E900090469946A246AB46F0BD5B463B430193F4
:107EA00000D12FE1002F00D1A5E1380000F0EEFD58
:107EB00003000B3B1C2B00DD96E11D22D31A5A4612
:107EC0000100DA405E4608398F4013008E403B4384
:107ED00001939C4B00271B1A994600239B467DE784
:107EE000414653460B4393498C46E144002B00D056
:107EF0001AE102220220174300228CE7134300D12B
:107F00000DE14346002B00D181E1404600F0BEFD6B
:107F100002000B3A1C2A00DD72E1010043460839D9
:107F20008B4098461D239A1A5346D3401A00434665
:107F3000134352468A404946081A82498946814479
:107F4000002068E77B4B002700268EE7140C120404
:107F5000120C1100370C3604350C794328008C467E
:107F60002E0060436044834656432100300C804617
:107F70005846794340440291844506D98846802179
:107F800049028C46E044414602913604010C360C0D
:107F900000048B4681191E0C1B041B0C0391190055
:107FA00079438C46280075436544A8465843050C20
:107FB00045447743A94203D9802149028C4667444E
:107FC000290C8C4639000004000C2D042D18614446
:107FD000AB4405915946049101990F043F0C080CDC
:107FE000390051434243904602008C46090C8B46AF
:107FF00062437C4344445C44A04503D98021490248
:1080000088464244210C884661460904090C8C4686
:1080100039005943434370437E430F0CF618240440
:10802000BE19644442448C46B34203D980235B02A8
:1080300098464044029B61469846049B370443445B
:108040009B46AB45AD416B420D0405992D0C8C460A
:108050007F196744FD18A8465D462D19A542A44125
:1080600093466442A446C344DC448F42BF419845D2
:108070009B4193459241A445A4415B427F421F43EB
:10808000360C52426442BF192243BF186246381868
:108090004302D20D039913436A020A43501E8241E0
:1080A0006146ED0D2A434E023243D90100D4B3E0BC
:1080B0000126500832400243DE0732435B08224C5F
:1080C0005444002C62DD510709D00F2010400428D1
:1080D00005D0101D9042924152429B180200D901D6
:1080E00004D580241948E4000340544418488442CD
:1080F00000DD27E75E075B02D2081F0B630516430E
:108100005B0DB2E6002399460133042700269B4607
:1081100064E60323019781460C279B465EE6012215
:1081200001201743002276E6032303201F43434622
:1081300071E6C046FF07000001FCFFFFE0AE000053
:10814000FFFF0F800DFCFFFFFF030000FFFFFFFE9E
:10815000FE0700000023802700933F030026434BC7
:1081600083E6019B3200A446584670E6AC466EE6B4
:10817000802701993F0339422DD03B422BD11F4329
:108180003F033F0B00951600384B6EE601252D1B73
:10819000382D00DD66E61F2D40DC35481C005044BC
:1081A000160082408440EE40501E82413443144306
:1081B000EB40620709D00F222240042A05D022009A
:1081C000141D9442804140421B181A023ED50123DF
:1081D0000027002649E68027019B3F031F433F03FA
:1081E0003F0B0094214B40E603005A46283B9A403F
:1081F000002601926DE6584600F048FC203057E614
:1082000003005246283B9A401300002293E6504652
:1082100000F03CFC20307BE6CA4650E71F201E00E1
:108220004042041BE640202D03D0124C5444A3408E
:108230001A43501E8241324307260027164009D0B8
:108240000F200023104014000428B9D122005E073B
:108250005B021F0BD2081643002306E680273F036C
:108260001F433F033F0B1600004BFEE5FF070000D6
:108270001E0400003E040000F8B557464E46454631
:10828000DE460C000903E0B5490A460F5F003143A2
:108290001E03DB0F760A9B46530F3343C84E65001F
:1082A000C000E40FD2006D0DA24681467F0D9C46B2
:1082B0009046B74200D1B9E05B46012673409B4629
:1082C000EE1BA34500D183E0002E63DD002F00D01C
:1082D000B1E06346134300D123E1731E002B00D0AD
:1082E000BAE1861A6346B04280410125C91A40426C
:1082F000091A0B0200D447E149024B0A984643464B
:10830000002B00D189E1404600F0C0FB0300083B90
:108310001F2B00DD7CE120223000D21A4146D040E4
:10832000994002009E400A439D4200DD6AE15D1BC8
:108330006B1C1F2B00DD94E1202110003500C91AB1
:108340008E40DA408840DD40711E8E4111000722C8
:108350002843002506433240002A09D00F2333402A
:10836000042B05D0331DB342B641764289191E0055
:108370000B0200D43DE26A1C914B55056D0D9A42EB
:1083800000D119E18F4AF6080A40570752023743D5
:10839000120B9BE0002E00D0C5E06E1C7605760D1A
:1083A000012E00DC48E16746861ACB1BB042BF4174
:1083B0007F42B8461F004346FF1A3B00B8461B02E7
:1083C00000D55FE137439AD100220024002579E0EF
:1083D000002E00DCFAE0002F00D18DE0784B9D42AA
:1083E00067D0802367461B041F43BC46382E00DC41
:1083F00052E1634613435A1E93411E188642804140
:10840000404209180B0200D4BEE06D4B01359D427D
:1084100000D1D2E06B4A73080A4001210E401E438E
:108420005108D30707221E43324095E71E0016432A
:1084300000D045E740E7624B9D423AD08023674633
:108440001B041F43BC46382E00DDEBE01F2E00DC72
:108450003AE133006746203BDF403B00202E05D049
:108460004027BF1B6646BE40324390464646721EBA
:1084700096413343DAE0002B00D114E26346134304
:1084800000D168E180234E07C008C9081B030643DA
:10849000194208D06046C008184204D16346010062
:1084A000D2085E071643F3009946C900720F444D87
:1084B00011434B46DE08424B4F073743CA089D42E3
:1084C00000D16EE012036D05120B6D0D0021120339
:1084D000130B0A0D12051A433B4B2D0513402B437A
:1084E0005B00E4075B082343380019003CBC90465E
:1084F0009946A246AB46F8BD6346134311D0731E9E
:10850000002B00D007E1861886428041614440423A
:10851000091801250B0237D502257BE73E0061468D
:1085200091463500C5E75C46002D00D0E1E00B0028
:108530000343F3D0731C00D1ACE1214B9F4200D127
:108540003AE1F343382B00DD6FE11F2B00DD8CE1B6
:1085500020250E00ED1AAE40B0460600AA46DE40C9
:10856000454635432E005546D940A8406346451E32
:10857000A8415B1A9C463043161AB24292416346A8
:108580005242991A3D00B4E607223240002A00D038
:10859000E4E60B4BF6084F073743CA089D4200D06C
:1085A00090E73B00134300D1A6E180231B031A434D
:1085B0001203120B024D89E715000022002785E700
:1085C000FF070000FFFF7FFFFFFF0F80002E00D09E
:1085D000C7E06B1C5E05760D012E00DCF0E0C84D97
:1085E000AB4200D1B9E085180A0085428941624456
:1085F000494251180722CE076D082E4349083240E0
:108600001D00A9E6BF49ED1A114007223240A3E63A
:10861000320028388240002686E6300000F036FA24
:10862000203073E6634613435A1E9341C61AB04284
:1086300080414042091A5CE60E0067460643174334
:10864000002D5ED1002E00D0F3E0002F00D11EE1FE
:108650005C46614691462CE7A94FBE427BD01E0086
:10866000F1E610001F3DE840202B03D04021CB1A3B
:108670009A401643731E9E41072206433240002152
:10868000002583E7161A6346B2428041591A4042D8
:108690000B1A98465C4632E61F2E00DDABE0202721
:1086A000BB1B9A4663465746BB40994613004F464C
:1086B000F3401F433B005746BA40571EBA4113438D
:1086C0006246F240891898E62027BB1B9A4663460B
:1086D0005746BB40994613004F46F3401F433B00AB
:1086E0005746BA40571EBA4113436246F240891AB0
:1086F0009CE7834B9F425FD080252D047342294322
:1087000020E7002E0CD1002F00D1D0E05C4661465E
:1087100091467B4DCDE67A4FBE421CD01E0065E6E9
:10872000002F18D0C0084E0706438020C908000358
:10873000014208D06346DC08044204D12100DA4635
:10874000D2085E071643F300994601245346C90038
:10875000720F11431C406A4DABE61D00002200273A
:10876000B4E6002D59D10B00034300D1D6E6731CAB
:1087700000D1B2E0624B9F421ED0F343382B6FDC36
:108780001F2B00DD97E020250E00ED1AAE40B0460D
:108790000600AA46DE40454635432E005546A84011
:1087A000D940451EA8418C440643B61896429241D2
:1087B000514261443D0025E63D006146914678E620
:1087C0000B000343002D00D055E6002BF5D0634687
:1087D000134300D16DE686188642804161444042D1
:1087E000091800220B0200D4D0E6464B013519408F
:1087F000B2E5B1465DE633006746203BDF403B0013
:10880000202E05D04027BF1B6646BE40324390460F
:108810004646721E96413343EFE5394B9F42CBD01B
:1088200080252D0473422943A8E70843411E88414F
:10883000A2E6002F00D13CE66346861ACF1AB0426A
:108840009B415B42FB1A98461B024ED5161A6346A3
:10885000B2429241591A5242891A5C4600227BE583
:1088600001430E00711E8E419FE71D000E00203D4A
:10887000EE40B046202B04D04025EB1A9940084327
:10888000814648464346411E8841184374E600220B
:10889000002417E6161A6346B2429241591A524210
:1088A000891A3D0025E561469146154D01E6802275
:1088B0000024120379E61D000E00203DEE40B04674
:1088C000202B04D04025EB1A9940084381464E46A0
:1088D0004346711E8E411E4367E7861896429B41B0
:1088E00061445B42C9183D008CE547463743CED012
:1088F00007224146324049E600273A00E6E5C046F5
:10890000FF070000FFFF7FFF30B5144D0A034B0047
:10891000120B5B0DC90F0024AB4211DD104CA342BA
:1089200010DC8024640322430E4CE41A1F2C0CDD5F
:108930000D48C31ADA4013005C42002900D11C0024
:10894000200030BD094BCC18FAE7094DE040AC4699
:1089500063449A4013000343EEE7C046FE03000061
:108960001D0400003304000013040000FFFFFF7F1C
:10897000EDFBFFFF70B500282DD0C317C5185D4073
:10898000C40F280000F082F8154B1B1A5B055B0D25
:108990000A2815DD0B38854000222D032D0B002100
:1089A00010002D030A0D2D0B12052A430D4D1B053A
:1089B0002A4013435B00E4075B082343190070BDA2
:1089C00002002900153291400A000B21081AC54007
:1089D0002D032D0BE3E70024002300250022DEE712
:1089E0001E040000FFFF0F804100090E4B1C70B5F4
:1089F000DBB24602750AC40F012B14DDE0239B0095
:108A00006D07360BCB1800210A0D280012051C4DEE
:108A100032435B052A405B0813435B00E4075B08B5
:108A20002343190070BD002914D1002D1ED0280049
:108A300000F02CF80A281CDC0B232A001B1ADA4051
:108A4000030015339D400F4B12031B1A5B05160BD9
:108A50005B0DD8E7002D06D0320B802636036D075C
:108A60001643094BCFE7084B0026CCE7002300262E
:108A7000C9E703002A000B3B9A400025E3E7C04604
:108A8000FFFF0F8089030000FF0700001C21012366
:108A90001B04984201D3000C10391B0A984201D3E1
:108AA000000A08391B09984201D30009043902A2BF
:108AB000105C40187047C046040302020101010126
:108AC000000000000000000030B51C00094B05004C
:108AD0001B6885B0D868084B002A01D1074B1A00E3
:108AE0000292019300912B002200054900F020F82A
:108AF00000F0FAFD3C02002020AF000043A400007B
:108B00002DAF0000084B10B50400002B02D000214F
:108B100000E000BF054B1868836A002B00D098471F
:108B2000200001F005FBC046000000005CAF000023
:108B30000EB403B5010003AB044804CB00680193F5
:108B400000F020F902B008BC03B018473C02002036
:108B500070B500260C4D0D4C641BA410A64209D123
:108B6000002601F0E7FA0A4D0A4C641BA410A64245
:108B700005D170BDB300EB5898470136EEE7B3005E
:108B8000EB5898470136F2E70C0400200C04002053
:108B90000C0400201C04002010B5034B01001868D1
:108BA00000F06AF810BDC0463C02002010B5034B2F
:108BB0000100186800F016F810BDC0463C02002005
:108BC000002310B59A4200D110BDCC5CC4540133CF
:108BD000F8E703001218934200D17047197001336F
:108BE000F9E7000070B50500002910D00C1F2368BC
:108BF000002B00DAE418280000F0A8FF1D4A1368D3
:108C0000002B05D163601460280000F0A0FF70BD48
:108C1000A34209D9216860188342F3D118685B68C0
:108C200041182160EEE713005A68002A01D0A242E1
:108C3000F9D919685818A0420BD12068091858189A
:108C400019608242E0D110685268411819605A6078
:108C5000DAE7A04202D90C232B60D5E7216860181F
:108C6000824203D1106852684118216062605C60E2
:108C7000CAE7C046E4130020032370B5CD1C9D4312
:108C8000083506000C2D1ED20C25A9421DD8300037
:108C900000F05CFF254A14682100002919D1244CFA
:108CA0002368002B03D1300000F02AFB206029004C
:108CB000300000F025FB431C2BD10C233000336027
:108CC00000F045FF03E0002DDFDA0C2333600020C5
:108CD00070BD0B685B1B19D40B2B03D90B60CC1830
:108CE000256003E04B688C420DD11360300000F02A
:108CF0002EFF200007220B30231D9043C31AE7D01C
:108D00005A42E250E4E763600C00EFE70C00496868
:108D1000C3E70323C41C9C43A042E1D0211A3000C6
:108D200000F0EEFA431CDBD1C7E7C046E413002095
:108D3000E8130020936810B5013B9360002B04DA20
:108D40009469A34207DB0A2905D01368581C1060F8
:108D50001970080010BD00F0FBFB0100F9E7F8B541
:108D600006000F001400D518AC4201D1002007E026
:108D700021783A003000FFF7DDFF0134431CF3D1C6
:108D8000F8BD0000F0B59FB002900F0016000593EB
:108D9000002805D083690493002B01D100F0A4FDC5
:108DA0007B4B9F425BD1029B5F68BB891B0762D5EF
:108DB0003B69002B5FD0002306AC636120336376F0
:108DC0001033A37635002B78002B01D0252B5CD1F6
:108DD000AB1B04930CD0320039000298FFF7BFFFA1
:108DE000431C00D1C4E06269049B94466344636100
:108DF0002B78002B00D1BBE001220023524262609D
:108E000002A9543252186E1C2360E360A3601370F1
:108E1000A365317805225F4800F07AFE751C0028B2
:108E200035D12268D30604D5532302A95B1820212B
:108E30001970130704D5532302A95B182B2119704D
:108E400033782A2B2CD0350000210A20E3682A78B9
:108E50006E1C303A092A64D900292ED026E04E4BE8
:108E60009F4202D1029B9F689FE74C4B9F429CD13F
:108E7000029BDF6899E73900029800F0BFFB0028E9
:108E800099D0012040421FB0F0BD01359BE7414B16
:108E90002268C01A01238340134323602E00B8E7E1
:108EA000059B191D1B680591002B01DB099304E04C
:108EB0005B42E3600223134323602B782E2B0AD1FD
:108EC0006B782A2B35D1059B02351A1D1B6805923C
:108ED000002B2BDB0793324E29780322300000F061
:108EE00017FE002806D04023801B834022680135EE
:108EF00013432360297806222A486E1C217600F04D
:108F000007FE00283AD0284B002B25D10722059BCD
:108F100007339343083305936369039A9B1863618E
:108F200050E7434301219B18350090E701235B4242
:108F3000D0E700230A201A000135636029786E1CEF
:108F40003039092903D9002BC5D00792C3E7424322
:108F5000012352183500F1E705AB00933A00134B9B
:108F60002100029800E000BF0390039B0133D3D19E
:108F7000BB895B0600D584E70B9884E705AB0093BB
:108F80003A000A4B2100029800F080F8ECE7C04656
:108F9000B4AF000060AF0000D4AF000094AF000099
:108FA00066AF00006AAF0000000000005F8D0000A7
:108FB000F7B5150001938A680B6900900C00934285
:108FC00000DA130022002B6043321278002A01D00D
:108FD00001332B6023689B0602D52B6802332B607C
:108FE000062723681F4027D0230043331B785A1ECF
:108FF00093412268920630D42200019943320098AE
:10900000089EB047431C25D0062320682A68E168E3
:1090100003400025042B03D18D1AEB43DB171D40C1
:10902000A3682269934201DD9B1AED180027BD4217
:1090300020D1002010E00137E3682A689B1ABB4268
:10904000D2DD22000123193201990098089EB04711
:10905000431CF0D101204042FEBD3020E1184331D5
:10906000087021005A1C45310978A2184332023396
:109070001170C1E7220001231A3201990098089E5D
:10908000B047431CE6D00137D1E70000F0B589B006
:1090900004920A0043320593039002920A7E0C0068
:1090A0000E9B6E2A00D186E01FD8632A33D008D8E1
:1090B000002A00D18CE0582A4DD0250042352A7074
:1090C00030E0642A01D0692AF7D1196825680A1DA1
:1090D000280629D508681A60002803DA2D23029A89
:1090E000404213706B4E0A274FE0732A74D008D8A1
:1090F0006F2A1FD0702AE0D1202209680A4322601B
:1091000003E0752A16D0782AD7D12200782145327B
:109110001170614E22E025001A684235111D196058
:1091200013682B70012365E008681A606906D3D5BF
:1091300000B2D1E719682568081D186008682E0676
:1091400005D5544E08276F2A1BD00A2719E06D0653
:10915000F7D580B2F5E745314E4E0A70186822689F
:10916000011D00681960150621D5D30702D52023FB
:109170001A4322601027002803D1202322689A4333
:1091800022602300002243331A706368A360002B1F
:1091900058DB0422216891432160002854D1029DAC
:1091A000002B5AD02500337842352B7055E05506F8
:1091B000DBD580B2D9E71A680D68101D49691860BF
:1091C00013682E0601D5196002E06D06FBD51980E3
:1091D0000023029D23614FE01A68111D1960156874
:1091E00000216268280000F093FC002801D0401B99
:1091F0006060636823610023029A13703CE0236976
:109200002A0004990398059DA847431C3ED0236873
:109210009B0715D4079BE068984239DA180037E0BD
:1092200022000123193204990398059EB047431C7C
:109230002CD00135E368079A9B1AAB42F0DCE9E7D2
:109240000025F7E70028ADD0029D3900FDF79CFE10
:10925000735C013D2B700028F7D1082F09D12368DA
:10926000DB0706D563682269934202DC3023013DA7
:109270002B70029B5B1B2361059B07AA00932100B7
:10928000049B0398FFF794FE431CB8D10120404291
:1092900009B0F0BD71AF000082AF0000124B10B5F5
:1092A0001C68A36B002B0FD11820FFF775FC0F4B28
:1092B000A06303600E4B012243600E4B83600B23BF
:1092C0008381002302614361A46B0B4A20696169B9
:1092D0000A4BFDF795FF01220023801859412061B8
:1092E00061614800400810BD3C0200200E33CDAB48
:1092F00034126DE6ECDE05002D7F954C2DF45158AF
:10930000002370B5064C05000800236000F0FAFE4B
:10931000431C03D12368002B00D02B6070BDC046D6
:10932000002800200CB430B5164B9DB00C1E1D68F3
:1093300008DA8B2301202B6040421DB030BC08BCF2
:1093400002B01847822302A99B008B810023029060
:1093500008619C4200D0631E8B604B6101235B421D
:10936000CB81209A21AB2800019300F079FC431CAB
:1093700001DA8B232B60002CDFD00023029A1370BC
:10938000DBE7C0463C0200200EB400B50B499CB0A0
:109390001DAB02900690079104910948094904CB3E
:1093A0000591006802A9019300F05AFC0023029A7B
:1093B00013701CB008BC03B01847C046FFFFFF7F06
:1093C0003C0200200802FFFF02780B78002A03D03D
:1093D000013001319A42F7D0D01A704703000A7861
:1093E00001311A700133002AF9D170470023C25CA1
:1093F0000133002AFBD1581E704730B50500002A02
:1094000000D130BD0C78013A6B1C2C700131002C5E
:1094100005D19A189A42F4D01C700133FAE71D0066
:10942000EDE70000F0B51F000E0087B00590019138
:1094300002920C98347800F0EAFA08220019437876
:10944000751C134036D12D2C36D1B51C74780126ED
:10945000002F62D0102F09D1302C07D120222B7879
:109460009343582B54D110276C7802352D4B39007B
:10947000F31818000393FDF787FD049101210023E1
:10948000494202008C4618002100303909291AD8B7
:109490000C00A74223DD591C09D06346824206D343
:1094A00002D10499A14202DB0123784320182C78D1
:1094B0000135E9E72E00BCE72B2C01D01E00C7E7E1
:1094C000B51C7478FAE721004139192901D8373CD5
:1094D000DFE721006139192901D8573CD9E75A1C27
:1094E00008D1059A23331360029B0398002B09D1FE
:1094F00007B0F0BD002E00D04042029A002AF7D0FB
:10950000002B01D06B1E0193029B019A1A60EFE7BA
:109510003024002FAAD10827A8E7302C9ED00A2794
:10952000A4E7C046FFFFFF7F37B51300064A0500DA
:109530001068046A002C00D1044C0A000094290031
:10954000FFF770FF3EBDC0463C020020A002002095
:10955000F8B505000E001400002804D08369002B24
:1095600001D100F0C1F9224B9C422DD16C68A36956
:10957000A360A3891B0731D52369002B2ED0236854
:109580002269F7B2981A6369F6B2834205DC2100BA
:10959000280000F03BF9002826D1A3680130013BE8
:1095A000A36023685A1C22601F706369834204D041
:1095B000A389DB071AD50A2E18D12100280000F054
:1095C00025F9002812D00FE00A4B9C4201D1AC686B
:1095D000CDE7094B9C42CAD1EC68C8E721002800BE
:1095E00000F00CF80028CAD0012676423000F8BD01
:1095F000B4AF0000D4AF000094AF0000364B70B59C
:109600001D6806000C00002D05D0AB69002B02D1AF
:10961000280000F069F9314B9C420FD16C680C2393
:10962000E25E93B219072DD4D90611D40923012083
:10963000336037331343A381404270BD284B9C42B3
:1096400001D1AC68EBE7274B9C42E8D1EC68E6E738
:109650005B0713D5616B002908D02300443399427E
:1096600002D03000FFF7BEFA002363632422A389EF
:109670009343A38100236360236923600823A289A5
:109680001343A3812369002B0BD1A0218022A3893E
:10969000890092000B40934203D02100300000F07B
:1096A000E1F90123A289134011D00023A36063696B
:1096B0005B42A361002023698342BED10C23E25E9A
:1096C0001306BAD540231343A3810138B5E79207A7
:1096D00000D46369A360EDE73C020020B4AF000052
:1096E000D4AF000094AF000010B5062000F0E0FBFE
:1096F000012000F01DFD0000F7B58A8905000C006F
:10970000130760D44B68002B04DC0B6C002B01DCCE
:109710000020FEBDE76A002FFAD000232E682B60E0
:1097200080235B01216A1A4034D0606DA3895B07F6
:1097300006D56368C01A636B002B01D0236CC01A76
:109740000200216A00232800E76AB847A189431C68
:1097500006D12B681D2B30D82B4ADA40D3072CD5E5
:109760000023636023692360CB0405D5431C02D129
:109770002B68002B00D16065616B2E600029C7D07B
:1097800023004433994202D02800FFF72BFA00202F
:109790006063BEE701232800B847431CC6D12B688D
:1097A000002BC3D01D2B01D0162B01D12E60AFE7AB
:1097B0004023A2891343A381ABE740230B4301203D
:1097C000A3814042A5E70F69002FA1D00B680F606D
:1097D000DB1B01930023920700D14B69A360019B1F
:1097E000002B00DC94E7019B3A00216A2800A66A5E
:1097F000B047002803DC4023A2891343DFE7019B25
:109800003F181B1A0193EAE7010040200B6970B56D
:1098100005000C00002B01D1002070BD002804D0F1
:109820008369002B01D100F05FF80B4B9C4209D1FA
:109830006C680C22A35E002BEED021002800FFF7FD
:109840005BFFEAE7054B9C4201D1AC68F1E7044BB2
:109850009C42EED1EC68ECE7B4AF0000D4AF00005E
:1098600094AF0000002310B50400036043608360E0
:1098700081814366C28103614361836119000822CB
:109880005C30FFF7A6F9054B24626362044BA362C8
:10989000044BE362044B236310BDC046F19E0000FD
:1098A000199F0000519F00007D9F000010B50249E4
:1098B00000F08CF810BDC0460D98000070B568250A
:1098C0004A1E55430E0029007431FFF7D5F9041ED6
:1098D00008D000212A00016046600C30A060683288
:1098E000FFF777F9200070BD836913B50400002BE2
:1098F00028D18364C3640365134B144A1B688262D6
:109900000193984201D101238361200000F020F8E7
:109910006060200000F01CF8A060200000F018F843
:109920000022E06004216068FFF79CFF012209210A
:10993000A068FFF797FF02221221E068FFF792FF6D
:109940000123A36113BDC0465CAF0000AD980000C9
:10995000F8B51C4B07001E68B369002B02D130001C
:10996000FFF7C2FF4836B4687368013B04D533681B
:10997000002B07D03668F6E70C22A55E002D0DD02F
:109980006834F2E704213800FFF798FF30600028C0
:10999000F0D10C2304003B602000F8BD20000A4BEE
:1099A000656625606560A560E36025616561A56108
:1099B000082229005C30FFF70CF96563A563A564F4
:1099C000E564E9E75CAF00000100FFFFF7B50400C4
:1099D0000700002601914834002C01D13000FEBD63
:1099E0006368A5680093009B013B009301D5246840
:1099F000F2E7AB89012B08D90E22AB5E013304D00C
:109A000029003800019B984706436835EBE7EC30A6
:109A10000068704770B50E001D000E23C95E96B039
:109A20001400002907DA00232B60B3891B0611D428
:109A30008023DB000FE06A4600F0D8FA0028F2DB52
:109A4000F022019B12021340054A9B185A425341CF
:109A50002B60EDE740230020236016B070BDC046A8
:109A600000E0FFFFF7B502268B8905000C003342AA
:109A700006D0230047332360236101236361F7BDD0
:109A800001AB6A46FFF7C6FF009907002800FFF701
:109A9000F3F8002808D10C22A35E9A05EFD4032224
:109AA00093431E43A681E4E70F4BAB628023A28958
:109AB00020601343A381009B20616361019B002B05
:109AC0000DD00E23E15E280000F0A2FA002806D097
:109AD0000322A38993431A0001231343A381A0897E
:109AE0003843A081CBE7C046AD98000082B0002982
:109AF00000D101A9101E06D0002B06D013780B60F0
:109B00001078431E984102B0704702204042FAE7A5
:109B1000C9B28218904201D10020704703788B426D
:109B2000FBD00130F6E710B5884202D98B18984275
:109B300003D3002307E08B5C8354013AFBD210BDB2
:109B4000CC5CC45401339A42FAD1F8E770477047AD
:109B5000F8B507000D001600002905D11100FFF728
:109B60008BF804002000F8BD002A03D1FFF73AF873
:109B70003400F7E700F072FA2C00B042F2D2310064
:109B80003800FFF779F8041EECD029003200FFF707
:109B900017F829003800FFF725F8E3E7F0B58E68DD
:109BA00085B007000C00039201939E423CD890239D
:109BB0008A89DB001A4234D00325096923685B1ABD
:109BC0000293636902985D43EB0F5D19019B6D1071
:109BD00001331B18AB4200D91D00530532D52900B3
:109BE0003800FFF749F8061E09D10C233B604023DB
:109BF0000120A28940421343A38105B0F0BD029A1F
:109C00002169FEF7DDFFA389144A1A40802313431C
:109C1000A381029B2661F61826606561019EED1AFC
:109C2000A560019B9E4200D9019E320003992068E5
:109C3000FFF779FFA36800209B1BA36023689E1990
:109C40002660DAE72A003800FFF782FF061EE0D11F
:109C500021693800FEF7C6FFC7E7C0467FFBFFFF5C
:109C6000F0B59FB0029005938B890F0016001B067C
:109C700011D50B69002B0ED14021FEF7FDFF386096
:109C80003861002805D10C23029A013813601FB0F7
:109C9000F0BD40237B61002306AC63612033637613
:109CA0001033A37635002B78002B01D0252B46D11D
:109CB000AB1B04930CD0320039000298FFF76EFF03
:109CC000431C00D1AEE06269049B94466344636127
:109CD0002B78002B00D1A5E00122002352426260C4
:109CE00002A9543252186E1C2360E360A360137003
:109CF000A365317805225448FFF70AFF751C002838
:109D00001FD12268D30604D5532302A95B18202152
:109D10001970130704D5532302A95B182B2119705E
:109D200033782A2B16D0350000210A20E3682A78E0
:109D30006E1C303A092A4ED9002918D010E001359E
:109D4000B1E7414B2268C01A0123834013432360CB
:109D50002E00CEE7059B191D1B680591002B01DB2A
:109D6000099304E05B42E3600223134323602B78F2
:109D70002E2B0AD16B782A2B35D1059B02351A1D63
:109D80001B680592002B2BDB0793304E29780322AA
:109D90003000FFF7BDFE002806D04023801B834023
:109DA00022680135134323602978062228486E1C57
:109DB0002176FFF7ADFE00283CD0264B002B25D1A5
:109DC0000722059B07339343083305936369039A7E
:109DD0009B18636166E7434301219B183500A6E7A2
:109DE00001235B42D0E700230A201A00013563609B
:109DF00029786E1C3039092903D9002BC5D0079268
:109E0000C3E74243012352183500F1E705AB009345
:109E10003A00114B2100029800E000BF0390039B21
:109E20000133D3D1BB890B985B0600D42FE7012007
:109E300040422CE705AB00933A00074B2100029803
:109E4000FFF724F9EAE7C04660AF000066AF000004
:109E50006AAF0000000000009D9B000070B5040088
:109E60000D001F2904D9162303600120404270BD54
:109E7000436C002B04D08A009B181A68002A08D172
:109E8000200000F031F82A000100200000F01AF84C
:109E9000EDE70020012AEAD0511C03D1162301303E
:109EA0002360E4E7002428001C6090472000DEE7E0
:109EB00010B5034B01001868FFF7D0FF10BDC04676
:109EC0003C020020002370B5064C0500080011007C
:109ED000236000F0FFF8431C03D12368002B00D05F
:109EE0002B6070BD0028002010B500F0E3F810BD15
:109EF00070B50C000E25495F00F0B8F8002803DBB0
:109F0000636D1B18636570BDA389024A1340A3816A
:109F1000F9E7C046FFEFFFFFF8B51F008B8905008A
:109F20000C001600DB0505D50E23C95E00220223B6
:109F300000F080F8A389054A28001340A38132006D
:109F40000E23E15E3B0000F02BF8F8BDFFEFFFFFB2
:109F500070B50C000E25495F00F06CF8A389421C17
:109F600003D1054A1340A38170BD802252011343DF
:109F7000A3816065F8E7C046FFEFFFFF10B50E2331
:109F8000C95E00F021F810BD0B1E04D0FF2A04D9D1
:109F90008A2303608B3B180070470A700123FAE79D
:109FA00070B50500080011000022064C22601A005E
:109FB00000F0B6F8431C03D12368002B00D02B60BF
:109FC00070BDC04600280020002370B5064C050077
:109FD0000800236000F05EF8431C03D12368002BC7
:109FE00000D02B6070BDC04600280020002370B553
:109FF000064C050008001100236000F053F8431CD4
:10A0000003D12368002B00D02B6070BD00280020F6
:10A01000002370B5064C05000800236000F052F8DC
:10A02000431C03D12368002B00D02B6070BDC046B9
:10A030000028002070B50500080011000022064C21
:10A0400022601A0000F04EF8431C03D12368002B55
:10A0500000D02B6070BDC046002800200B1F1B687D
:10A06000181F002B01DA0B58C018704770B5050097
:10A07000080011000022064C22601A0000F03AF895
:10A08000431C03D12368002B00D02B6070BDC04659
:10A090000028002058220120014B40421A607047DE
:10A0A0000028002058220120014B40421A607047CE
:10A0B0000028002058220120014B40421A607047BE
:10A0C000002800205822024B00201A607047C0462A
:10A0D0000028002058220120014B40421A6070479E
:10A0E0000028002058220120014B40421A6070478E
:10A0F0000028002058220120014B40421A6070477E
:10A1000000280020044A1368002B00D1034B1818C4
:10A11000106018007047C046EC130020082800208B
:10A1200058220120014B40421A607047002800204D
:10A13000FEE7C046F8B5C046F8BC08BC9E4670476E
:10A14000F8B5C046F8BC08BC9E46704750050000F4
:10A15000600500007A050000F805000030060000E8
:10A16000660600009E060000C4060000000700000E
:10A170004207000098070000DC07000048080000C4
:10A1800090080000B6080000EE0800003409000046
:10A190005A09000088090000BA090000F20900000D
:10A1A000760A0000420B0000B80B0000240C0000EF
:10A1B0006C0C00008C0C0000AE0C0000880D000040
:10A1C000CE0D0000500500005005000050050000B5
:10A1D000460E0000AE0E0000300F0000760F0000AB
:10A1E000BE0F00003C100000BA1000000211000079
:10A1F000481100007E110000C41100000A12000086
:10A2000052120000A61200000413000042130000C6
:10A21000AC130000E21300002A14000072140000C6
:10A22000BA140000F41400003C150000841500006E
:10A23000500500005005000050050000EC1500001E
:10A24000221600005816000084160000BA160000FE
:10A25000F0160000500500005005000050050000F9
:10A260005005000026170000681700005005000088
:10A2700050050000AE170000FE1700002418000073
:10A280005005000050050000500500005218000065
:10A2900082180000B2180000E21800000C1900003B
:10A2A000421900006C19000094190000BC1900004C
:10A2B000EC1900001C1A0000461A0000701A000079
:10A2C000A01A0000E41A000050050000500500002C
:10A2D000500500005005000050050000141B000050
:10A2E000401B00006C1B0000981B0000C41B0000FA
:10A2F000FA1B0000301C0000661C00009C1C0000C3
:10A30000C81C0000F41C00002A1D000050050000BD
:10A3100050050000500500005005000050050000E9
:10A3200050050000500500005005000050050000D9
:10A3300050050000500500005005000050050000C9
:10A3400050050000561D0000821D000066616C7300
:10A35000650074727565006C697374206F662025E2
:10A3600064206974656D73006F626A656374206F41
:10A370006620636C6173733A2025640053746163D3
:10A380006B20756E646572666C6F77000700000065
:10A3900003000000000000000100000002000000B7
:10A3A00003000000040000000A0000006D696372F1
:10A3B0006F3A62697400686173546F6E6500706C07
:10A3C0006179546F6E6500686173536572766F00D2
:10A3D000736574536572766F00496E73756666694E
:10A3E0006369656E74206D656D6F727920666F723A
:10A3F000204D6963726F426C6F636B73206F626A8A
:10A40000656374206865617000496E73756666697E
:10A410006369656E74206D656D6F727920666F7209
:10A42000204D6963726F426C6F636B73207374614C
:10A43000636B000D0A564D2050616E69633A20250A
:10A44000730D0A006D69736300686578546F496E17
:10A45000740073696E006E657400686173576946B5
:10A4600069007374617274576946690073746F7020
:10A47000576946690077696669537461747573003A
:10A480006D79495041646472657373007468696ED4
:10A49000674465736372697074696F6E00636C659D
:10A4A00061725468696E6744657363726970746938
:10A4B0006F6E00617070656E64546F5468696E678A
:10A4C0004465736372697074696F6E006170706562
:10A4D0006E64546F5468696E6750726F7065727401
:10A4E00079001A1B1C03040607090A17181903042C
:10A4F0000607090A171819000000000008080800DC
:10A50000080A4A4000000A5FEA5FEA0ED92ED36EBD
:10A5100019324489330C924C924D08080000000413
:10A52000880808040804848488000A448A400004D7
:10A530008EC480000000048800000EC000000000EF
:10A54000080001224488100C9252524C048C8484DE
:10A550008E1C824C901E1EC244924C06CA525FE270
:10A560001FF01EC13E02448ED12E1FE24488100E01
:10A57000D12ED12E0ED12EC4880008000800000470
:10A580008004880244880482000EC00EC008048241
:10A5900044880ED126C0040ED135B36C0C925ED225
:10A5A000521C925C925C0ED010100E1C9252525CA7
:10A5B0001ED01C901E1ED01C90100ED013712E1297
:10A5C000525ED2521C8808081C1FE242524C1254A0
:10A5D000981492101010101E113B75B131113935BD
:10A5E000B3710C9252524C1C925C90100C92524CD3
:10A5F000861C925C92510ED00C825C1FE484848491
:10A60000125252524C1131312A44113135BB711260
:10A61000524C9252112A4484841EC488101E0EC8C3
:10A6200008080E10080482410EC242424E048A40BD
:10A630000000000000001F0804800000000ED2523D
:10A640004F10101C925C000ED0100E02424ED24EE3
:10A650000C925C900E06C81C88080ED24EC24C109C
:10A66000101C92520800080808024002424C1014C4
:10A670009814920808080806001B75B131001C9256
:10A680005252000C92524C001C925C90000ED24E22
:10A69000C2000ED010100006C8049808080EC807A3
:10A6A000001252524F0011312A4400113135BB00C3
:10A6B000124C8C9200112A4498001EC4881E06C4B5
:10A6C0008C8486080808080818080C881800000CF4
:10A6D0008360000000000000010000000200000094
:10A6E0000300000004000000050000000600000058
:10A6F0000700000008000000090000000A00000038
:10A700000B0000000C0000000D0000000E00000017
:10A710000F000000100000001200000014000000F4
:10A7200016000000180000001A0000001C000000C5
:10A730001E00000020000000230000002600000092
:10A74000290000002C0000002F0000003200000053
:10A75000360000003A0000003E0000004200000009
:10A76000460000004B0000005000000055000000B3
:10A770005A00000061000000680000006F00000047
:10A78000760000007D000000840000008B000000C7
:10A790009200000099000000A0000000A700000047
:10A7A000AE000000B5000000BC000000C3000000C7
:10A7B000CA000000D1000000D8000000DF00000047
:10A7C000E6000000ED000000F4000000FB000000C7
:10A7D000FF000000646973706C6179006C696768E0
:10A7E000744C6576656C006D62446973706C617958
:10A7F000006D62446973706C61794F6666006D62CA
:10A80000506C6F74006D62556E706C6F74006D6289
:10A81000447261775368617065006D62536861705E
:10A8200065466F724C6574746572006E656F506931
:10A8300078656C53656E64006E656F506978656C01
:10A8400053657450696E004E6F7420656E6F756746
:10A850006820726F6F6D206576656E206166746525
:10A860007220636F6D70616374696F6E0A00436F6D
:10A870006D70616374656420466C61736820636FFA
:10A8800064652073746F72650A256420627974654B
:10A8900073207573656420282564252529206F663B
:10A8A00020256400426164207265636F72642066D3
:10A8B0006F756E6420647572696E6720696E697465
:10A8C00069616C697A6174696F6E210A0025642080
:10A8D00025642025642028256420776F72647329FD
:10A8E000002564207265636F7264732C20256420D8
:10A8F000776F7264732C206D617849442025642C35
:10A9000020636F6D70616374696F6E206379636C2F
:10A910006573202564005363726970747320636CDF
:10A920006561726564005374617274656400526598
:10A9300073746F7265642025642073637269707428
:10A940007300726164696F006E756D626572006E8E
:10A950006F6E65006F746865720070616972007374
:10A960007472696E670064697361626C65526164D8
:10A97000696F006D657373616765526563656976BC
:10A980006564007061636B657452656365697665C3
:10A99000007061636B657453656E64007265636516
:10A9A00069766564496E7465676572007265636592
:10A9B000697665644D657373616765547970650088
:10A9C0007265636569766564537472696E67007356
:10A9D000656E64496E74656765720073656E645078
:10A9E0006169720073656E64537472696E67007397
:10A9F00065744368616E6E656C0073657447726F51
:10AA0000757000736574506F776572007369676E57
:10AA1000616C537472656E67746800416C6C20746D
:10AA200061736B732073746F707065640076303679
:10AA30003500202573202573004D656D6F727920D8
:10AA4000636C6561726564004E6F20667265652097
:10AA50007461736B20656E74726965730073656EE3
:10AA6000736F72730074656D706572617475726571
:10AA70000074696C74580074696C74590074696C62
:10AA8000745A00746F75636852656164006932635B
:10AA90005265616400693263577269746500746657
:10AAA0007400656E61626C65446973706C617900F5
:10AAB0006765745769647468006765744865696799
:10AAC000687400736574506978656C006C696E65B4
:10AAD000007265637400726F756E646564526563BD
:10AAE0007400636972636C6500747269616E676C8F
:10AAF00065007465787400746674546F7563686576
:10AB00006400746674546F75636858007466745496
:10AB10006F7563685900746674546F75636850721A
:10AB20006573737572650057656C636F6D6520742E
:10AB30006F204D6963726F426C6F636B732100709D
:10AB40005F73706920213D204E554C4C002F686F7B
:10AB50006D652F62726F6D61676F73612F2E706C00
:10AB60006174666F726D696F2F7061636B61676589
:10AB7000732F6672616D65776F726B2D617264758C
:10AB8000696E6F6E6F726469636E7266352F6C6981
:10AB9000627261726965732F5350492F5350492E69
:10ABA00063707000535049436C6173733A3A535069
:10ABB00049436C617373284E52465F5350495F544A
:10ABC0007970652A2C2075696E74385F742C207535
:10ABD000696E74385F742C2075696E74385F7429DF
:10ABE000000000000000000000000000894D00008F
:10ABF000454D00006B4D0000754D00007F4D00007D
:10AC0000694D000003000000020000000100000088
:10AC10000400000005000000110000000C0000000E
:10AC20000B000000120000000A00000006000000F7
:10AC30001A000000140000001700000016000000B9
:10AC40001500000010000000FFFFFFFFFFFFFFFFE7
:10AC5000000000001E0000001900000018000000A5
:10AC60000700000008000000090000000D000000BF
:10AC70000E0000000F0000001C0000001B00000080
:10AC80001D00000013000000000000000000000094
:10AC90009152000075500000115300002553000030
:10ACA0001B5300008D520000815200003153000000
:10ACB000AD5200007D520000000000000000304353
:10ACC00000000000000030C3FB21F93FFB210940D8
:10ACD0007CD91240FB2119407A6A1F407CD922405E
:10ACE000BBFD2540FB2129403A462C407A6A2F4083
:10ACF0005C4731407CD932409C6B3440BBFD3540D1
:10AD0000DB8F3740FB2139401BB43A403A463C4088
:10AD10005AD83D407A6A3F404C7E40405C474140B3
:10AD20006C1042407CD942408CA243409C6B444012
:10AD3000AC344540BBFD4540CBC64640DB8F474069
:10AD4000EB584840FB21494083F9A200444E6E0075
:10AD5000FC291500D1572700DD34F50062DBC00067
:10AD60003C999500419043006351FE00BBDEAB006F
:10AD7000B761C5003A6E2400D24D42004906E0009A
:10AD800009EA2E001C92D100EB1DFE0029B11C0027
:10AD9000E83EA700F535820044BB2E009CE9840004
:10ADA000B4267000417E5F00D6913900538339008C
:10ADB0009CF439008B5F840028F9BD00F81F3B002C
:10ADC000DEFF97000F980500112FEF000A5A8B0045
:10ADD0006D1F6D00CF7E360009CB2700464FB700B0
:10ADE0009E663F002DEA5F00BA277500E5EBC700BD
:10ADF0003D7BF100F739070092528A00FB6BEA00B5
:10AE00001FB15F00085D8D00300356007BFC4600DB
:10AE1000F0AB6B0020BCCF0036F49A00E3A91D0014
:10AE20005E619100081BE60085996500A0145F0033
:10AE30008D40680080D8FF0027734D000606310062
:10AE4000CA561500C9A873007BE260006B8CC00075
:10AE500000000040FB21F93F000000002D44743E3B
:10AE6000000000809846F83C0000006051CC783B20
:10AE700000000080831BF0390000004020257A3854
:10AE8000000000802282E336000000001DF36935D7
:10AE900002000000030000000400000006000000A3
:10AEA0004C730000F6720000F6720000247400007B
:10AEB000F2720000F27200001A74000024740000A4
:10AEC000F27200001A740000F27200002474000094
:10AED00028740000287400002874000030740000FA
:10AEE0004C7F00004E7E00004E7E00006C81000012
:10AEF000487E0000487E0000548100006C81000004
:10AF0000487E000054810000487E00006C810000F3
:10AF10006281000062810000628100007081000097
:10AF20002C2066756E6374696F6E3A2000617373CE
:10AF3000657274696F6E2022257322206661696CC8
:10AF400065643A2066696C6520222573222C206C8A
:10AF5000696E65202564257325730A004002002070
:10AF6000232D302B2000686C4C00656667454647F2
:10AF70000030313233343536373839414243444575
:10AF800046003031323334353637383961626364E4
:10AF900065660000000000000000000000000000E6
:10AFA00000000000000000000000000000000000A1
:10AFB0000000000000000000000000000000000091
:10AFC0000000000000000000000000000000000081
:10AFD0000000000000000000000000000000000071
:10AFE0000000000000000000000000000000000061
:10AFF000000000004300504F534958002E0000202D
:10B000002020202020202020282828282820202018
:10B0100020202020202020202020202020202088C8
:10B02000101010101010101010101010101010042C
:10B03000040404040404040404101010101010107C
:10B040004141414141410101010101010101010170
:10B050000101010101010101010110101010101086
:10B060004242424242420202020202020202020240
:10B07000020202020202020202021010101020005C
:10B0800000000000000000000000000000000000C0
:10B0900000000000000000000000000000000000B0
:10B0A00000000000000000000000000000000000A0
:10B0B0000000000000000000000000000000000090
:10B0C0000000000000000000000000000000000080
:10B0D0000000000000000000000000000000000070
:10B0E0000000000000000000000000000000000060
:10B0F0000000000000000000000000000000000050
:04B10000000000004B
:08B104000450FF7F0100000070
:10B10C00FFFFFFFF40060000B6A300005D1E00001D
:10B11C00BEA30000611E0000C7A30000591E000062
:10B12C00D0A30000651E000049A40000A12200006D
:10B13C0052A40000F52200005AA40000D123000004
:10B14C0062A40000D52300006CA40000F3230000CF
:10B15C0075A40000FD23000080A40000072400005B
:10B16C008CA40000112400009DA400001B240000EE
:10B17C00B3A40000DF230000CCA40000E9230000EE
:10B18C00DCA7000041240000E7A700000D29000007
:10B19C00F1A7000021260000FEA7000041260000B8
:10B1AC0005A80000912600000EA80000E126000072
:10B1BC001AA80000392900002BA800005128000013
:10B1CC0038A80000212800001800000066A9000023
:10B1DC007933000073A90000D935000083A9000061
:10B1EC007D35000091A90000593700009CA9000092
:10B1FC0091330000ACA90000F9330000C0A9000095
:10B20C00A1330000CFA9000039390000DBA90000F0
:10B21C00B9380000E4A900005D380000EFA9000077
:10B22C00A5370000FAA90000E137000003AA0000CE
:10B23C00153800000CAA0000A933000019FCFFFF10
:10B24C00FFFFFFFF65AA00003147000071AA000054
:10B25C00994A000077AA0000A94A00007DAA0000C4
:10B26C00B94A000083AA0000654700008DAA0000BF
:10B27C00C94A000095AA0000A5480000FF00000084
:10B28C00A2AA00004D4B0000B0AA0000594B0000D0
:10B29C00B9AA00005D4B0000C3AA0000614B00007E
:10B2AC00CCAA0000654B0000D1AA0000694B00003D
:10B2BC00D6AA00006D4B0000E2AA0000714B000002
:10B2CC00E9AA0000754B0000F2AA0000794B0000BF
:10B2DC00F7AA00007D4B000002AB0000814B000080
:10B2EC000CAB0000514B000016AB0000554B00009E
:10B2FC000200000003000000FFFFFFFF0000000041
:10B30C00010000000000020001000000FFFFFFFF31
:10B31C000000000002000000000004000200000019
:10B32C00FFFFFFFF0000000003000000000008000A
:10B33C00030000000A00000008000000400200208A
:10B34C0000000000B4AF0000D4AF000094AF0000C8
:10B35C0000000000000000000000000000000000E1
:10B36C0000000000000000000000000000000000D1
:10B37C0000000000000000000000000000000000C1
:10B38C0000000000000000000000000000000000B1
:10B39C0000000000000000000000000000000000A1
:10B3AC00430000000000000000000000000000004E
:10B3BC000000000000000000000000000000000081
:10B3CC00430000000000000000000000000000002E
:10B3DC000000000000000000000000000000000061
:10B3EC00430000000000000000000000000000000E
:10B3FC000000000000000000000000000000000041
:10B40C0043000000000000000000000000000000ED
:10B41C000000000000000000000000000000000020
:10B42C0043000000000000000000000000000000CD
:10B43C000000000000000000000000000000000000
:10B44C0043000000000000000000000000000000AD
:10B45C0000000000000000000000000000000000E0
:10B46C00430000000000000000000000000000008D
:10B47C0000000000000000000000000000000000C0
:10B48C00899F0000ED9A000000000000FEAF000054
:10B49C00FCAF000043A4000043A4000043A4000040
:10B4AC0043A4000043A4000043A4000043A40000F4
:10B4BC0043A4000043A40000FFFFFFFFFFFFFFFFBA
:10B4CC00FFFFFFFFFFFF000001004153434949000C
:10B4DC000000000000000000000000000000000060
:10B4EC0000000000000000000000415343494900E7
:10B4FC000000000000000000000000000000000040
:10B50C00000000000000000000000000E900000046
:10B51C00154D00005D500000DD550000C10000001D
:040000030000515157
:00000001FF
